 thrcputime002

 Timestamp is 9a3a69fb (reproducible build file hash)

 Preferred load address is 0000000180000000

 Start         Length     Name                   Class
 0001:00000000 00004370H .text$mn                CODE
 0001:00004370 00000036H .text$mn$00             CODE
 0001:000043a6 00000092H .text$x                 CODE
 0002:00000000 000001c8H .idata$5                DATA
 0002:000001c8 00000038H .00cfg                  DATA
 0002:00000200 00000008H .CRT$XCA                DATA
 0002:00000208 00000008H .CRT$XCZ                DATA
 0002:00000210 00000008H .CRT$XIA                DATA
 0002:00000218 00000008H .CRT$XIC                DATA
 0002:00000220 00000008H .CRT$XIZ                DATA
 0002:00000228 00000008H .CRT$XLA                DATA
 0002:00000230 00000008H .CRT$XLZ                DATA
 0002:00000238 00000008H .CRT$XPA                DATA
 0002:00000240 00000008H .CRT$XPZ                DATA
 0002:00000248 00000008H .CRT$XTA                DATA
 0002:00000250 00000010H .CRT$XTZ                DATA
 0002:00000258 00000000H .gehcont$y              DATA
 0002:00000258 00000000H .gfids$y                DATA
 0002:00000260 00002820H .rdata                  DATA
 0002:00002a80 00000000H .rdata$CastGuardVftablesA DATA
 0002:00002a80 00000000H .rdata$CastGuardVftablesC DATA
 0002:00002a80 00000028H .rdata$T                DATA
 0002:00002aa8 000000bcH .rdata$voltmd           DATA
 0002:00002b64 0000031cH .rdata$zzzdbg           DATA
 0002:00002e80 00000008H .rtc$IAA                DATA
 0002:00002e88 00000008H .rtc$IZZ                DATA
 0002:00002e90 00000008H .rtc$TAA                DATA
 0002:00002e98 00000008H .rtc$TZZ                DATA
 0002:00002ea0 00000004H .tls                    DATA
 0002:00002ea4 00000004H .tls$                   DATA
 0002:00002ea8 00000008H .tls$ZZZ                DATA
 0002:00002eb0 000003f0H .xdata                  DATA
 0002:000032a0 000003d4H .edata                  DATA
 0002:00003674 0000008cH .idata$2                DATA
 0002:00003700 00000018H .idata$3                DATA
 0002:00003718 000001c8H .idata$4                DATA
 0002:000038e0 00000486H .idata$6                DATA
 0003:00000000 00000090H .data                   DATA
 0003:00000090 0001b258H .bss                    DATA
 0004:00000000 00000444H .pdata                  DATA

  Address         Publics by Value              Rva+Base               Lib:Object

 0000:00000000       __AbsoluteZero             0000000000000000     <absolute>
 0000:00000000       ___safe_se_handler_count   0000000000000000     <absolute>
 0000:00000000       ___safe_se_handler_table   0000000000000000     <absolute>
 0000:00000000       __arm64x_extra_rfe_table   0000000000000000     <absolute>
 0000:00000000       __arm64x_extra_rfe_table_size 0000000000000000     <absolute>
 0000:00000000       __arm64x_native_entrypoint 0000000000000000     <absolute>
 0000:00000000       __arm64x_redirection_metadata 0000000000000000     <absolute>
 0000:00000000       __arm64x_redirection_metadata_count 0000000000000000     <absolute>
 0000:00000000       __dynamic_value_reloc_table 0000000000000000     <absolute>
 0000:00000000       __enclave_config           0000000000000000     <absolute>
 0000:00000000       __guard_check_icall_a64n_fptr 0000000000000000     <absolute>
 0000:00000000       __guard_eh_cont_count      0000000000000000     <absolute>
 0000:00000000       __guard_eh_cont_table      0000000000000000     <absolute>
 0000:00000000       __guard_fids_count         0000000000000000     <absolute>
 0000:00000000       __guard_fids_table         0000000000000000     <absolute>
 0000:00000000       __guard_iat_count          0000000000000000     <absolute>
 0000:00000000       __guard_iat_table          0000000000000000     <absolute>
 0000:00000000       __guard_longjmp_count      0000000000000000     <absolute>
 0000:00000000       __guard_longjmp_table      0000000000000000     <absolute>
 0000:00000000       __hybrid_auxiliary_iat     0000000000000000     <absolute>
 0000:00000000       __hybrid_auxiliary_iat_copy 0000000000000000     <absolute>
 0000:00000000       __hybrid_code_map          0000000000000000     <absolute>
 0000:00000000       __hybrid_code_map_count    0000000000000000     <absolute>
 0000:00000000       __x64_code_ranges_to_entry_points 0000000000000000     <absolute>
 0000:00000000       __x64_code_ranges_to_entry_points_count 0000000000000000     <absolute>
 0000:00000100       __guard_flags              0000000000000100     <absolute>
 0000:00000000       __ImageBase                0000000180000000     <linker-defined>
 0001:00000000       ?NewObject@JNIEnv_@@QEAAPEAV_jobject@@PEAV_jclass@@PEAU_jmethodID@@ZZ 0000000180001000 f i libthrcputime002.obj
 0001:00000028       ?SetEventNotificationMode@_jvmtiEnv@@QEAA?AW4jvmtiError@@W4jvmtiEventMode@@W4jvmtiEvent@@PEAV_jobject@@ZZ 0000000180001028 f i libthrcputime002.obj
 0001:00000034       ?TranslateError@@YAPEBDW4jvmtiError@@@Z 0000000180001034 f   libthrcputime002.obj
 0001:00000354       ?create_raw_monitor@@YAPEAU_jrawMonitorID@@PEAU_jvmtiEnv@@PEBD@Z 0000000180001354 f   libthrcputime002.obj
 0001:00000380       ?julong_to_string@@YAPEAD_KPEAD@Z 0000000180001380 f   libthrcputime002.obj
 0001:00000410       ?nsk_jni_check_exception@@YAHPEAUJNIEnv_@@QEBDH@Z 0000000180001410 f   libthrcputime002.obj
 0001:00000554       ?nsk_jni_lverify@@YAHHPEAUJNIEnv_@@HQEBDH1ZZ 0000000180001554 f   libthrcputime002.obj
 0001:000005f4       Agent_Initialize           00000001800015f4 f   libthrcputime002.obj
 0001:0000099c       Agent_OnAttach             000000018000199c f   libthrcputime002.obj
 0001:0000099c       Agent_OnLoad               000000018000199c f   libthrcputime002.obj
 0001:000009a4       Java_nsk_jvmti_unit_FollowReferences_FollowRefObjects_addRefToVerify 00000001800019a4 f   libthrcputime002.obj
 0001:00000b7c       Java_nsk_jvmti_unit_FollowReferences_FollowRefObjects_getTag 0000000180001b7c f   libthrcputime002.obj
 0001:00000c3c       Java_nsk_jvmti_unit_FollowReferences_FollowRefObjects_resetRefsToVerify 0000000180001c3c f   libthrcputime002.obj
 0001:00000c44       Java_nsk_jvmti_unit_FollowReferences_FollowRefObjects_resetTags 0000000180001c44 f   libthrcputime002.obj
 0001:00000c88       Java_nsk_jvmti_unit_FollowReferences_FollowRefObjects_setTag 0000000180001c88 f   libthrcputime002.obj
 0001:00000ee0       Java_nsk_share_jvmti_ArgumentHandler_getAgentOptionsString 0000000180001ee0 f   libthrcputime002.obj
 0001:00000f90       Java_nsk_share_jvmti_DebugeeClass_checkStatus 0000000180001f90 f   libthrcputime002.obj
 0001:00001018       Java_nsk_share_jvmti_DebugeeClass_resetAgentData 0000000180002018 f   libthrcputime002.obj
 0001:00001078       Java_nsk_share_jvmti_RedefineAgent_agentStatus 0000000180002078 f   libthrcputime002.obj
 0001:00001084       Java_nsk_share_jvmti_RedefineAgent_isRedefined 0000000180002084 f   libthrcputime002.obj
 0001:00001090       Java_nsk_share_jvmti_RedefineAgent_redefineAttempted 0000000180002090 f   libthrcputime002.obj
 0001:0000109c       MA_checkStatus             000000018000209c f   libthrcputime002.obj
 0001:00001140       __local_stdio_printf_options 0000000180002140 f i libthrcputime002.obj
 0001:000016d4       callbackThreadEnd          00000001800026d4 f   libthrcputime002.obj
 0001:00001914       callbackThreadStart        0000000180002914 f   libthrcputime002.obj
 0001:00001b5c       callbackVMDeath            0000000180002b5c f   libthrcputime002.obj
 0001:00001c68       callbackVMInit             0000000180002c68 f   libthrcputime002.obj
 0001:00002144       exitOnError                0000000180003144 f   libthrcputime002.obj
 0001:000021f8       fprintf                    00000001800031f8 f i libthrcputime002.obj
 0001:0000223c       nsk_complain               000000018000323c f   libthrcputime002.obj
 0001:00002268       nsk_jvmti_createJVMTIEnv   0000000180003268 f   libthrcputime002.obj
 0001:00002398       nsk_jvmti_enableEvents     0000000180003398 f   libthrcputime002.obj
 0001:0000246c       nsk_jvmti_findOptionIntValue 000000018000346c f   libthrcputime002.obj
 0001:00002508       nsk_jvmti_findOptionValue  0000000180003508 f   libthrcputime002.obj
 0001:00002580       nsk_jvmti_lverify          0000000180003580 f   libthrcputime002.obj
 0001:00002670       nsk_jvmti_parseOptions     0000000180003670 f   libthrcputime002.obj
 0001:000028c0       nsk_jvmti_resetAgentData   00000001800038c0 f   libthrcputime002.obj
 0001:00002940       nsk_jvmti_resumeSync       0000000180003940 f   libthrcputime002.obj
 0001:000029e8       nsk_jvmti_setFailStatus    00000001800039e8 f   libthrcputime002.obj
 0001:00002a24       nsk_jvmti_waitForSync      0000000180003a24 f   libthrcputime002.obj
 0001:00002b28       nsk_lcomplain              0000000180003b28 f   libthrcputime002.obj
 0001:00002b48       nsk_ldisplay               0000000180003b48 f   libthrcputime002.obj
 0001:00002b68       nsk_ltrace                 0000000180003b68 f   libthrcputime002.obj
 0001:00002b88       nsk_lvcomplain             0000000180003b88 f   libthrcputime002.obj
 0001:00002d40       nsk_lvdisplay              0000000180003d40 f   libthrcputime002.obj
 0001:00002d8c       nsk_lverify                0000000180003d8c f   libthrcputime002.obj
 0001:00002de8       nsk_lvtrace                0000000180003de8 f   libthrcputime002.obj
 0001:00002e48       nsk_printf                 0000000180003e48 f   libthrcputime002.obj
 0001:00002e70       nsk_vprintf                0000000180003e70 f   libthrcputime002.obj
 0001:00002f24       printf                     0000000180003f24 f i libthrcputime002.obj
 0001:0000344c       __raise_securityfailure    000000018000444c f   MSVCRT:gs_report.obj
 0001:00003480       __report_gsfailure         0000000180004480 f   MSVCRT:gs_report.obj
 0001:000036c0       __GSHandlerCheck           00000001800046c0 f   MSVCRT:gshandler.obj
 0001:000036e0       __GSHandlerCheckCommon     00000001800046e0 f   MSVCRT:gshandler.obj
 0001:00003750       __security_check_cookie    0000000180004750 f   MSVCRT:amdsecgs.obj
 0001:00003a90       _DllMainCRTStartup         0000000180004a90 f   MSVCRT:dll_dllmain.obj
 0001:00003ad0       __scrt_acquire_startup_lock 0000000180004ad0 f   MSVCRT:utility.obj
 0001:00003b0c       __scrt_dllmain_after_initialize_c 0000000180004b0c f   MSVCRT:utility.obj
 0001:00003b40       __scrt_dllmain_before_initialize_c 0000000180004b40 f   MSVCRT:utility.obj
 0001:00003b58       __scrt_dllmain_crt_thread_attach 0000000180004b58 f   MSVCRT:utility.obj
 0001:00003b80       __scrt_dllmain_crt_thread_detach 0000000180004b80 f   MSVCRT:utility.obj
 0001:00003b98       __scrt_dllmain_exception_filter 0000000180004b98 f   MSVCRT:utility.obj
 0001:00003bf8       __scrt_dllmain_uninitialize_c 0000000180004bf8 f   MSVCRT:utility.obj
 0001:00003c28       __scrt_dllmain_uninitialize_critical 0000000180004c28 f   MSVCRT:utility.obj
 0001:00003c3c       __scrt_initialize_crt      0000000180004c3c f   MSVCRT:utility.obj
 0001:00003c88       __scrt_initialize_onexit_tables 0000000180004c88 f   MSVCRT:utility.obj
 0001:00003d14       __scrt_is_nonwritable_in_current_image 0000000180004d14 f   MSVCRT:utility.obj
 0001:00003dac       __scrt_release_startup_lock 0000000180004dac f   MSVCRT:utility.obj
 0001:00003dd0       __scrt_uninitialize_crt    0000000180004dd0 f   MSVCRT:utility.obj
 0001:00003dfc       _onexit                    0000000180004dfc f   MSVCRT:utility.obj
 0001:00003e38       atexit                     0000000180004e38 f   MSVCRT:utility.obj
 0001:00003e50       __crt_debugger_hook        0000000180004e50 f   MSVCRT:utility_desktop.obj
 0001:00003e58       __scrt_fastfail            0000000180004e58 f   MSVCRT:utility_desktop.obj
 0001:00003fa4       _guard_check_icall_nop     0000000180004fa4 f i MSVCRT:guard_support.obj
 0001:00003fa8       __security_init_cookie     0000000180004fa8 f   MSVCRT:gs_support.obj
 0001:00004054       DllMain                    0000000180005054 f   MSVCRT:dll_dllmain_stub.obj
 0001:00004078       ?__scrt_initialize_type_info@@YAXXZ 0000000180005078 f   MSVCRT:tncleanup.obj
 0001:00004088       ?__scrt_uninitialize_type_info@@YAXXZ 0000000180005088 f   MSVCRT:tncleanup.obj
 0001:00004094       __local_stdio_scanf_options 0000000180005094 f i MSVCRT:default_local_stdio_options.obj
 0001:0000409c       __scrt_initialize_default_local_stdio_options 000000018000509c f   MSVCRT:default_local_stdio_options.obj
 0001:000040b8       __scrt_get_dyn_tls_init_callback 00000001800050b8 f   MSVCRT:dyn_tls_init.obj
 0001:000040c0       _RTC_Initialize            00000001800050c0 f   MSVCRT:initsect.obj
 0001:000040fc       _RTC_Terminate             00000001800050fc f   MSVCRT:initsect.obj
 0001:00004138       __isa_available_init       0000000180005138 f   MSVCRT:cpu_disp.obj
 0001:000042e4       _get_startup_argv_mode     00000001800052e4 f   MSVCRT:argv_mode.obj
 0001:000042ec       __scrt_is_ucrt_dll_in_use  00000001800052ec f   MSVCRT:ucrt_detection.obj
 0001:00004300       memcpy                     0000000180005300 f   vcruntime:VCRUNTIME140.dll
 0001:00004306       memset                     0000000180005306 f   vcruntime:VCRUNTIME140.dll
 0001:0000430c       strchr                     000000018000530c f   vcruntime:VCRUNTIME140.dll
 0001:00004312       __C_specific_handler       0000000180005312 f   vcruntime:VCRUNTIME140.dll
 0001:00004318       __std_type_info_destroy_list 0000000180005318 f   vcruntime:VCRUNTIME140.dll
 0001:0000431e       strcmp                     000000018000531e f   ucrt:api-ms-win-crt-string-l1-1-0.dll
 0001:00004324       strlen                     0000000180005324 f   ucrt:api-ms-win-crt-string-l1-1-0.dll
 0001:0000432a       _initterm                  000000018000532a f   ucrt:api-ms-win-crt-runtime-l1-1-0.dll
 0001:00004330       _initterm_e                0000000180005330 f   ucrt:api-ms-win-crt-runtime-l1-1-0.dll
 0001:00004336       _seh_filter_dll            0000000180005336 f   ucrt:api-ms-win-crt-runtime-l1-1-0.dll
 0001:0000433c       _configure_narrow_argv     000000018000533c f   ucrt:api-ms-win-crt-runtime-l1-1-0.dll
 0001:00004342       _initialize_narrow_environment 0000000180005342 f   ucrt:api-ms-win-crt-runtime-l1-1-0.dll
 0001:00004348       _initialize_onexit_table   0000000180005348 f   ucrt:api-ms-win-crt-runtime-l1-1-0.dll
 0001:0000434e       _register_onexit_function  000000018000534e f   ucrt:api-ms-win-crt-runtime-l1-1-0.dll
 0001:00004354       _execute_onexit_table      0000000180005354 f   ucrt:api-ms-win-crt-runtime-l1-1-0.dll
 0001:0000435a       _crt_atexit                000000018000535a f   ucrt:api-ms-win-crt-runtime-l1-1-0.dll
 0001:00004360       _cexit                     0000000180005360 f   ucrt:api-ms-win-crt-runtime-l1-1-0.dll
 0001:00004368       __acrt_initialize          0000000180005368 f   MSVCRT:ucrt_stubs.obj
 0001:00004368       __acrt_thread_attach       0000000180005368 f   MSVCRT:ucrt_stubs.obj
 0001:00004368       __acrt_thread_detach       0000000180005368 f   MSVCRT:ucrt_stubs.obj
 0001:00004368       __acrt_uninitialize        0000000180005368 f   MSVCRT:ucrt_stubs.obj
 0001:00004368       __acrt_uninitialize_critical 0000000180005368 f   MSVCRT:ucrt_stubs.obj
 0001:00004368       __scrt_stub_for_acrt_initialize 0000000180005368 f   MSVCRT:ucrt_stubs.obj
 0001:00004368       __scrt_stub_for_acrt_thread_attach 0000000180005368 f   MSVCRT:ucrt_stubs.obj
 0001:00004368       __scrt_stub_for_acrt_thread_detach 0000000180005368 f   MSVCRT:ucrt_stubs.obj
 0001:00004368       __scrt_stub_for_acrt_uninitialize 0000000180005368 f   MSVCRT:ucrt_stubs.obj
 0001:00004368       __scrt_stub_for_acrt_uninitialize_critical 0000000180005368 f   MSVCRT:ucrt_stubs.obj
 0001:00004368       __vcrt_initialize          0000000180005368 f   MSVCRT:ucrt_stubs.obj
 0001:00004368       __vcrt_thread_attach       0000000180005368 f   MSVCRT:ucrt_stubs.obj
 0001:00004368       __vcrt_thread_detach       0000000180005368 f   MSVCRT:ucrt_stubs.obj
 0001:00004368       __vcrt_uninitialize        0000000180005368 f   MSVCRT:ucrt_stubs.obj
 0001:00004368       __vcrt_uninitialize_critical 0000000180005368 f   MSVCRT:ucrt_stubs.obj
 0001:0000436c       __scrt_stub_for_is_c_termination_complete 000000018000536c f   MSVCRT:ucrt_stubs.obj
 0001:0000436c       _is_c_termination_complete 000000018000536c f   MSVCRT:ucrt_stubs.obj
 0001:00004380       _guard_dispatch_icall_nop  0000000180005380 f   MSVCRT:guard_dispatch.obj
 0001:000043a0       _guard_xfg_dispatch_icall_nop 00000001800053a0 f   MSVCRT:guard_xfg_dispatch.obj
 0002:00000000       __imp_RtlCaptureContext    0000000180006000     kernel32:KERNEL32.dll
 0002:00000008       __imp_RtlLookupFunctionEntry 0000000180006008     kernel32:KERNEL32.dll
 0002:00000010       __imp_RtlVirtualUnwind     0000000180006010     kernel32:KERNEL32.dll
 0002:00000018       __imp_UnhandledExceptionFilter 0000000180006018     kernel32:KERNEL32.dll
 0002:00000020       __imp_SetUnhandledExceptionFilter 0000000180006020     kernel32:KERNEL32.dll
 0002:00000028       __imp_GetCurrentProcess    0000000180006028     kernel32:KERNEL32.dll
 0002:00000030       __imp_TerminateProcess     0000000180006030     kernel32:KERNEL32.dll
 0002:00000038       __imp_IsProcessorFeaturePresent 0000000180006038     kernel32:KERNEL32.dll
 0002:00000040       __imp_CloseHandle          0000000180006040     kernel32:KERNEL32.dll
 0002:00000048       __imp_InitializeCriticalSectionAndSpinCount 0000000180006048     kernel32:KERNEL32.dll
 0002:00000050       __imp_DeleteCriticalSection 0000000180006050     kernel32:KERNEL32.dll
 0002:00000058       __imp_CreateEventW         0000000180006058     kernel32:KERNEL32.dll
 0002:00000060       __imp_GetModuleHandleW     0000000180006060     kernel32:KERNEL32.dll
 0002:00000068       __imp_GetProcAddress       0000000180006068     kernel32:KERNEL32.dll
 0002:00000070       __imp_IsDebuggerPresent    0000000180006070     kernel32:KERNEL32.dll
 0002:00000078       __imp_QueryPerformanceCounter 0000000180006078     kernel32:KERNEL32.dll
 0002:00000080       __imp_GetCurrentProcessId  0000000180006080     kernel32:KERNEL32.dll
 0002:00000088       __imp_GetCurrentThreadId   0000000180006088     kernel32:KERNEL32.dll
 0002:00000090       __imp_GetSystemTimeAsFileTime 0000000180006090     kernel32:KERNEL32.dll
 0002:00000098       __imp_DisableThreadLibraryCalls 0000000180006098     kernel32:KERNEL32.dll
 0002:000000a0       __imp_InitializeSListHead  00000001800060a0     kernel32:KERNEL32.dll
 0002:000000a8       \177KERNEL32_NULL_THUNK_DATA 00000001800060a8     kernel32:KERNEL32.dll
 0002:000000b0       __imp_memcpy               00000001800060b0     vcruntime:VCRUNTIME140.dll
 0002:000000b8       __imp_memset               00000001800060b8     vcruntime:VCRUNTIME140.dll
 0002:000000c0       __imp_strchr               00000001800060c0     vcruntime:VCRUNTIME140.dll
 0002:000000c8       __imp___C_specific_handler 00000001800060c8     vcruntime:VCRUNTIME140.dll
 0002:000000d0       __imp___std_type_info_destroy_list 00000001800060d0     vcruntime:VCRUNTIME140.dll
 0002:000000d8       \177VCRUNTIME140_NULL_THUNK_DATA 00000001800060d8     vcruntime:VCRUNTIME140.dll
 0002:000000e0       __imp_strtol               00000001800060e0     ucrt:api-ms-win-crt-convert-l1-1-0.dll
 0002:000000e8       \177api-ms-win-crt-convert-l1-1-0_NULL_THUNK_DATA 00000001800060e8     ucrt:api-ms-win-crt-convert-l1-1-0.dll
 0002:000000f0       __imp_malloc               00000001800060f0     ucrt:api-ms-win-crt-heap-l1-1-0.dll
 0002:000000f8       __imp_free                 00000001800060f8     ucrt:api-ms-win-crt-heap-l1-1-0.dll
 0002:00000100       \177api-ms-win-crt-heap-l1-1-0_NULL_THUNK_DATA 0000000180006100     ucrt:api-ms-win-crt-heap-l1-1-0.dll
 0002:00000108       __imp__errno               0000000180006108     ucrt:api-ms-win-crt-runtime-l1-1-0.dll
 0002:00000110       __imp_exit                 0000000180006110     ucrt:api-ms-win-crt-runtime-l1-1-0.dll
 0002:00000118       __imp__cexit               0000000180006118     ucrt:api-ms-win-crt-runtime-l1-1-0.dll
 0002:00000120       __imp__crt_atexit          0000000180006120     ucrt:api-ms-win-crt-runtime-l1-1-0.dll
 0002:00000128       __imp__execute_onexit_table 0000000180006128     ucrt:api-ms-win-crt-runtime-l1-1-0.dll
 0002:00000130       __imp__register_onexit_function 0000000180006130     ucrt:api-ms-win-crt-runtime-l1-1-0.dll
 0002:00000138       __imp__initialize_onexit_table 0000000180006138     ucrt:api-ms-win-crt-runtime-l1-1-0.dll
 0002:00000140       __imp__initialize_narrow_environment 0000000180006140     ucrt:api-ms-win-crt-runtime-l1-1-0.dll
 0002:00000148       __imp__configure_narrow_argv 0000000180006148     ucrt:api-ms-win-crt-runtime-l1-1-0.dll
 0002:00000150       __imp__seh_filter_dll      0000000180006150     ucrt:api-ms-win-crt-runtime-l1-1-0.dll
 0002:00000158       __imp__initterm_e          0000000180006158     ucrt:api-ms-win-crt-runtime-l1-1-0.dll
 0002:00000160       __imp__initterm            0000000180006160     ucrt:api-ms-win-crt-runtime-l1-1-0.dll
 0002:00000168       \177api-ms-win-crt-runtime-l1-1-0_NULL_THUNK_DATA 0000000180006168     ucrt:api-ms-win-crt-runtime-l1-1-0.dll
 0002:00000170       __imp___acrt_iob_func      0000000180006170     ucrt:api-ms-win-crt-stdio-l1-1-0.dll
 0002:00000178       __imp_fflush               0000000180006178     ucrt:api-ms-win-crt-stdio-l1-1-0.dll
 0002:00000180       __imp___stdio_common_vsprintf 0000000180006180     ucrt:api-ms-win-crt-stdio-l1-1-0.dll
 0002:00000188       __imp___stdio_common_vfprintf 0000000180006188     ucrt:api-ms-win-crt-stdio-l1-1-0.dll
 0002:00000190       \177api-ms-win-crt-stdio-l1-1-0_NULL_THUNK_DATA 0000000180006190     ucrt:api-ms-win-crt-stdio-l1-1-0.dll
 0002:00000198       __imp_strcmp               0000000180006198     ucrt:api-ms-win-crt-string-l1-1-0.dll
 0002:000001a0       __imp__strdup              00000001800061a0     ucrt:api-ms-win-crt-string-l1-1-0.dll
 0002:000001a0       __imp_strdup               00000001800061a0     ucrt:api-ms-win-crt-string-l1-1-0.dll
 0002:000001a8       __imp_strlen               00000001800061a8     ucrt:api-ms-win-crt-string-l1-1-0.dll
 0002:000001b0       __imp_strpbrk              00000001800061b0     ucrt:api-ms-win-crt-string-l1-1-0.dll
 0002:000001b8       __imp_strncpy              00000001800061b8     ucrt:api-ms-win-crt-string-l1-1-0.dll
 0002:000001c0       \177api-ms-win-crt-string-l1-1-0_NULL_THUNK_DATA 00000001800061c0     ucrt:api-ms-win-crt-string-l1-1-0.dll
 0002:000001c8       __guard_check_icall_fptr   00000001800061c8     MSVCRT:guard_support.obj
 0002:000001d0       __guard_xfg_check_icall_fptr 00000001800061d0     MSVCRT:guard_support.obj
 0002:000001d8       __guard_dispatch_icall_fptr 00000001800061d8     MSVCRT:guard_support.obj
 0002:000001e0       __guard_xfg_dispatch_icall_fptr 00000001800061e0     MSVCRT:guard_support.obj
 0002:000001e8       __guard_xfg_table_dispatch_icall_fptr 00000001800061e8     MSVCRT:guard_support.obj
 0002:000001f0       __castguard_check_failure_os_handled_fptr 00000001800061f0     MSVCRT:guard_support.obj
 0002:000001f8       __guard_memcpy_fptr        00000001800061f8     vcruntime:softmemtag.obj
 0002:00000200       __xc_a                     0000000180006200     MSVCRT:initializers.obj
 0002:00000208       __xc_z                     0000000180006208     MSVCRT:initializers.obj
 0002:00000210       __xi_a                     0000000180006210     MSVCRT:initializers.obj
 0002:00000220       __xi_z                     0000000180006220     MSVCRT:initializers.obj
 0002:00000228       __xl_a                     0000000180006228     MSVCRT:tlssup.obj
 0002:00000230       __xl_z                     0000000180006230     MSVCRT:tlssup.obj
 0002:00000238       __xp_a                     0000000180006238     MSVCRT:initializers.obj
 0002:00000240       __xp_z                     0000000180006240     MSVCRT:initializers.obj
 0002:00000248       __xt_a                     0000000180006248     MSVCRT:initializers.obj
 0002:00000250       __xt_z                     0000000180006250     MSVCRT:initializers.obj
 0002:00000260       g_refKindStr               0000000180006260     libthrcputime002.obj
 0002:00000410       ??_C@_09BPLDFGCI@unknown_0@ 0000000180006410     libthrcputime002.obj
 0002:00000420       ??_C@_0BL@FPNMECJD@JVMTI_HEAP_REFERENCE_CLASS@ 0000000180006420     libthrcputime002.obj
 0002:00000440       ??_C@_0BL@FKGKKLNM@JVMTI_HEAP_REFERENCE_FIELD@ 0000000180006440     libthrcputime002.obj
 0002:00000460       ??_C@_0CD@CAEHCFJF@JVMTI_HEAP_REFERENCE_ARRAY_ELEM@ 0000000180006460     libthrcputime002.obj
 0002:00000488       ??_C@_0CC@DNEBMCNK@JVMTI_HEAP_REFERENCE_CLASS_LOAD@ 0000000180006488     libthrcputime002.obj
 0002:000004b0       ??_C@_0BN@CJMIPEBB@JVMTI_HEAP_REFERENCE_SIGNERS@ 00000001800064b0     libthrcputime002.obj
 0002:000004d0       ??_C@_0CH@HBOIDPEB@JVMTI_HEAP_REFERENCE_PROTECTION@ 00000001800064d0     libthrcputime002.obj
 0002:000004f8       ??_C@_0BP@MDKGDGKL@JVMTI_HEAP_REFERENCE_INTERFACE@ 00000001800064f8     libthrcputime002.obj
 0002:00000518       ??_C@_0CC@JJMIHNJH@JVMTI_HEAP_REFERENCE_STATIC_FIE@ 0000000180006518     libthrcputime002.obj
 0002:00000540       ??_C@_0CD@IDHEEGID@JVMTI_HEAP_REFERENCE_CONSTANT_P@ 0000000180006540     libthrcputime002.obj
 0002:00000568       ??_C@_0CA@EFFCHNG@JVMTI_HEAP_REFERENCE_SUPERCLASS@ 0000000180006568     libthrcputime002.obj
 0002:00000588       ??_C@_0L@PCDFHGCJ@unknown_11@ 0000000180006588     libthrcputime002.obj
 0002:00000598       ??_C@_0L@NJBICFOK@unknown_12@ 0000000180006598     libthrcputime002.obj
 0002:000005a8       ??_C@_0L@MAADBEKL@unknown_13@ 00000001800065a8     libthrcputime002.obj
 0002:000005b8       ??_C@_0L@IPECICGM@unknown_14@ 00000001800065b8     libthrcputime002.obj
 0002:000005c8       ??_C@_0L@JGFJLDCN@unknown_15@ 00000001800065c8     libthrcputime002.obj
 0002:000005d8       ??_C@_0L@LNHEOAOO@unknown_16@ 00000001800065d8     libthrcputime002.obj
 0002:000005e8       ??_C@_0L@KEGPNBKP@unknown_17@ 00000001800065e8     libthrcputime002.obj
 0002:000005f8       ??_C@_0L@CDPHMNGA@unknown_18@ 00000001800065f8     libthrcputime002.obj
 0002:00000608       ??_C@_0L@DKOMPMCB@unknown_19@ 0000000180006608     libthrcputime002.obj
 0002:00000618       ??_C@_0L@OJGIPJDB@unknown_20@ 0000000180006618     libthrcputime002.obj
 0002:00000628       ??_C@_0CA@KAOFNDEM@JVMTI_HEAP_REFERENCE_JNI_GLOBAL@ 0000000180006628     libthrcputime002.obj
 0002:00000648       ??_C@_0CC@HPFAJBK@JVMTI_HEAP_REFERENCE_SYSTEM_CLA@ 0000000180006648     libthrcputime002.obj
 0002:00000670       ??_C@_0BN@FDEGFOHC@JVMTI_HEAP_REFERENCE_MONITOR@ 0000000180006670     libthrcputime002.obj
 0002:00000690       ??_C@_0CB@HKIBCMAJ@JVMTI_HEAP_REFERENCE_STACK_LOCA@ 0000000180006690     libthrcputime002.obj
 0002:000006b8       ??_C@_0BP@EAACMMOE@JVMTI_HEAP_REFERENCE_JNI_LOCAL@ 00000001800066b8     libthrcputime002.obj
 0002:000006d8       ??_C@_0BM@IJDEOGOE@JVMTI_HEAP_REFERENCE_THREAD@ 00000001800066d8     libthrcputime002.obj
 0002:000006f8       ??_C@_0BL@EDGPPKC@JVMTI_HEAP_REFERENCE_OTHER@ 00000001800066f8     libthrcputime002.obj
 0002:00000714       ??_C@_04BCJPDBDA@Code@     0000000180006714     libthrcputime002.obj
 0002:00000720       ??_C@_0BA@OCLMCFKC@LineNumberTable@ 0000000180006720     libthrcputime002.obj
 0002:00000730       ??_C@_0BD@CPAEPILC@LocalVariableTable@ 0000000180006730     libthrcputime002.obj
 0002:00000748       ??_C@_0BH@NMBDNHBD@LocalVariableTypeTable@ 0000000180006748     libthrcputime002.obj
 0002:00000760       ??_C@_0O@HIHEEDNJ@StackMapTable@ 0000000180006760     libthrcputime002.obj
 0002:00000770       ??_C@_0L@HCDIAMJG@?9?5?$CFs?0?5?$CFd?3?5@ 0000000180006770     libthrcputime002.obj
 0002:00000780       ??_C@_0JI@HLPECLFI@?$CD?5?4?4?4?6?$CD?5ERROR?3?5too?5many?5complai@ 0000000180006780     libthrcputime002.obj
 0002:00000820       ??_C@_0ED@JNEKCCOB@The?5following?5fake?5exception?5st@ 0000000180006820     libthrcputime002.obj
 0002:00000868       ??_C@_0CN@FCNMDFBH@nsk?4share?4Fake_Exception_for_RU@ 0000000180006868     libthrcputime002.obj
 0002:00000898       ??_C@_08PGFFNAEI@?$CI?$CFs?3?$CFd?$CJ?5@ 0000000180006898     libthrcputime002.obj
 0002:000008a8       ??_C@_0DP@IENMAEGI@s?2test?2hotspot?2jtreg?2vmTestbase@ 00000001800068a8     libthrcputime002.obj
 0002:000008e8       ??_C@_0BL@NDJLFFJB@?7at?5nsk_lvcomplain?$CI?$CFs?3?$CFd?$CJ?6@ 00000001800068e8     libthrcputime002.obj
 0002:00000908       ??_C@_0BC@JOOKAFKF@?$CD?5ERROR?3?5?$CFs?0?5?$CFd?3?5@ 0000000180006908     libthrcputime002.obj
 0002:00000920       ??_C@_09KJEAHMEH@?$CD?5ERROR?3?5@ 0000000180006920     libthrcputime002.obj
 0002:0000092c       ??_C@_02GPIOPFAK@?$DO?$DO@ 000000018000692c     libthrcputime002.obj
 0002:00000930       ??_C@_02FODMEDOG@?$DM?$DM@ 0000000180006930     libthrcputime002.obj
 0002:00000934       ??_C@_02DJGKEECL@?4?4@     0000000180006934     libthrcputime002.obj
 0002:00000938       ??_C@_0O@CJPGJOAF@?9?5?$CFs?0?5?$CFd?3?5?$CFs?5@ 0000000180006938     libthrcputime002.obj
 0002:00000948       ??_C@_0CB@IAKPDOIC@?$CD?5?5?5verified?5assertion?5is?5FALSE@ 0000000180006948     libthrcputime002.obj
 0002:00000970       ??_C@_0CO@LGONDEPD@stdout?3?5fflush?5failed?5?9?5err?$DN?$CFd?5@ 0000000180006970     libthrcputime002.obj
 0002:000009a0       ??_C@_0CO@KBGKJPBD@stderr?3?5fflush?5failed?5?9?5err?$DN?$CFd?5@ 00000001800069a0     libthrcputime002.obj
 0002:000009d0       ??_C@_06HPGEIPLA@?$DMnull?$DO@ 00000001800069d0     libthrcputime002.obj
 0002:000009d8       ??_C@_0DM@KLJPMIDM@check_jvmti_status?3?5JVMTI?5funct@ 00000001800069d8     libthrcputime002.obj
 0002:00000a18       ??_C@_0CA@CCEFGCFD@Fatal?5Error?5in?5RawMonitorEnter?4@ 0000000180006a18     libthrcputime002.obj
 0002:00000a38       ??_C@_0BB@JCNMKLLK@JVMTI_ERROR_NONE@ 0000000180006a38     libthrcputime002.obj
 0002:00000a50       ??_C@_0BL@LDIMKLPH@JVMTI_ERROR_INVALID_THREAD@ 0000000180006a50     libthrcputime002.obj
 0002:00000a70       ??_C@_0CB@PJFPAIKJ@JVMTI_ERROR_INVALID_THREAD_GROU@ 0000000180006a70     libthrcputime002.obj
 0002:00000a98       ??_C@_0BN@LLMKHMNF@JVMTI_ERROR_INVALID_PRIORITY@ 0000000180006a98     libthrcputime002.obj
 0002:00000ab8       ??_C@_0CB@MBOFKAGB@JVMTI_ERROR_THREAD_NOT_SUSPENDE@ 0000000180006ab8     libthrcputime002.obj
 0002:00000ae0       ??_C@_0BN@FABOLPBI@JVMTI_ERROR_THREAD_SUSPENDED@ 0000000180006ae0     libthrcputime002.obj
 0002:00000b00       ??_C@_0BN@FDGNOBJM@JVMTI_ERROR_THREAD_NOT_ALIVE@ 0000000180006b00     libthrcputime002.obj
 0002:00000b20       ??_C@_0BL@GOBIFKNJ@JVMTI_ERROR_INVALID_OBJECT@ 0000000180006b20     libthrcputime002.obj
 0002:00000b40       ??_C@_0BK@FCMAJPPC@JVMTI_ERROR_INVALID_CLASS@ 0000000180006b40     libthrcputime002.obj
 0002:00000b60       ??_C@_0BP@IKLLBKEB@JVMTI_ERROR_CLASS_NOT_PREPARED@ 0000000180006b60     libthrcputime002.obj
 0002:00000b80       ??_C@_0BN@KLPPLKG@JVMTI_ERROR_INVALID_METHODID@ 0000000180006b80     libthrcputime002.obj
 0002:00000ba0       ??_C@_0BN@BCEKOKND@JVMTI_ERROR_INVALID_LOCATION@ 0000000180006ba0     libthrcputime002.obj
 0002:00000bc0       ??_C@_0BM@DFDGPME@JVMTI_ERROR_INVALID_FIELDID@ 0000000180006bc0     libthrcputime002.obj
 0002:00000be0       ??_C@_0BL@NELIEPEC@JVMTI_ERROR_NO_MORE_FRAMES@ 0000000180006be0     libthrcputime002.obj
 0002:00000c00       ??_C@_0BJ@BDBECFDM@JVMTI_ERROR_OPAQUE_FRAME@ 0000000180006c00     libthrcputime002.obj
 0002:00000c20       ??_C@_0BK@MIIFNLOB@JVMTI_ERROR_TYPE_MISMATCH@ 0000000180006c20     libthrcputime002.obj
 0002:00000c40       ??_C@_0BJ@HPCAOILC@JVMTI_ERROR_INVALID_SLOT@ 0000000180006c40     libthrcputime002.obj
 0002:00000c60       ??_C@_0BG@CHILOPNI@JVMTI_ERROR_DUPLICATE@ 0000000180006c60     libthrcputime002.obj
 0002:00000c78       ??_C@_0BG@DIEMLHKM@JVMTI_ERROR_NOT_FOUND@ 0000000180006c78     libthrcputime002.obj
 0002:00000c90       ??_C@_0BM@NHMCKHOB@JVMTI_ERROR_INVALID_MONITOR@ 0000000180006c90     libthrcputime002.obj
 0002:00000cb0       ??_C@_0BO@PPEDAJGL@JVMTI_ERROR_NOT_MONITOR_OWNER@ 0000000180006cb0     libthrcputime002.obj
 0002:00000cd0       ??_C@_0BG@FCAIPEID@JVMTI_ERROR_INTERRUPT@ 0000000180006cd0     libthrcputime002.obj
 0002:00000ce8       ??_C@_0CB@EGDBNKOI@JVMTI_ERROR_INVALID_CLASS_FORMA@ 0000000180006ce8     libthrcputime002.obj
 0002:00000d10       ??_C@_0CG@DGKOGIAL@JVMTI_ERROR_CIRCULAR_CLASS_DEFI@ 0000000180006d10     libthrcputime002.obj
 0002:00000d38       ??_C@_0BP@ICEALPKC@JVMTI_ERROR_FAILS_VERIFICATION@ 0000000180006d38     libthrcputime002.obj
 0002:00000d58       ??_C@_0DC@JDACLMIO@JVMTI_ERROR_UNSUPPORTED_REDEFIN@ 0000000180006d58     libthrcputime002.obj
 0002:00000d90       ??_C@_0DE@GKDKNOMJ@JVMTI_ERROR_UNSUPPORTED_REDEFIN@ 0000000180006d90     libthrcputime002.obj
 0002:00000dc8       ??_C@_0BO@LAFKIOG@JVMTI_ERROR_INVALID_TYPESTATE@ 0000000180006dc8     libthrcputime002.obj
 0002:00000de8       ??_C@_0DH@INDGCLLB@JVMTI_ERROR_UNSUPPORTED_REDEFIN@ 0000000180006de8     libthrcputime002.obj
 0002:00000e20       ??_C@_0DE@NHEOMMGI@JVMTI_ERROR_UNSUPPORTED_REDEFIN@ 0000000180006e20     libthrcputime002.obj
 0002:00000e58       ??_C@_0CA@EKPNJOEP@JVMTI_ERROR_UNSUPPORTED_VERSION@ 0000000180006e58     libthrcputime002.obj
 0002:00000e78       ??_C@_0BN@OFFMAHHL@JVMTI_ERROR_NAMES_DONT_MATCH@ 0000000180006e78     libthrcputime002.obj
 0002:00000e98       ??_C@_0DN@HHBBLAKE@JVMTI_ERROR_UNSUPPORTED_REDEFIN@ 0000000180006e98     libthrcputime002.obj
 0002:00000ed8       ??_C@_0DO@HMBGBGNA@JVMTI_ERROR_UNSUPPORTED_REDEFIN@ 0000000180006ed8     libthrcputime002.obj
 0002:00000f18       ??_C@_0BP@PBECGKHJ@JVMTI_ERROR_UNMODIFIABLE_CLASS@ 0000000180006f18     libthrcputime002.obj
 0002:00000f38       ??_C@_0BK@CANILEHF@JVMTI_ERROR_NOT_AVAILABLE@ 0000000180006f38     libthrcputime002.obj
 0002:00000f58       ??_C@_0CE@INJKMEFK@JVMTI_ERROR_MUST_POSSESS_CAPABI@ 0000000180006f58     libthrcputime002.obj
 0002:00000f80       ??_C@_0BJ@LBFPFPDM@JVMTI_ERROR_NULL_POINTER@ 0000000180006f80     libthrcputime002.obj
 0002:00000fa0       ??_C@_0BP@CHJPNNEM@JVMTI_ERROR_ABSENT_INFORMATION@ 0000000180006fa0     libthrcputime002.obj
 0002:00000fc0       ??_C@_0BP@OMFMNLC@JVMTI_ERROR_INVALID_EVENT_TYPE@ 0000000180006fc0     libthrcputime002.obj
 0002:00000fe0       ??_C@_0BN@BIBNPHHO@JVMTI_ERROR_ILLEGAL_ARGUMENT@ 0000000180006fe0     libthrcputime002.obj
 0002:00001000       ??_C@_0BK@KKNDHDCE@JVMTI_ERROR_NATIVE_METHOD@ 0000000180007000     libthrcputime002.obj
 0002:00001020       ??_C@_0BK@PMKCFHAE@JVMTI_ERROR_OUT_OF_MEMORY@ 0000000180007020     libthrcputime002.obj
 0002:00001040       ??_C@_0BK@NNJBDMNB@JVMTI_ERROR_ACCESS_DENIED@ 0000000180007040     libthrcputime002.obj
 0002:00001060       ??_C@_0BI@GHECLMNC@JVMTI_ERROR_WRONG_PHASE@ 0000000180007060     libthrcputime002.obj
 0002:00001078       ??_C@_0BF@OLIHJOII@JVMTI_ERROR_INTERNAL@ 0000000180007078     libthrcputime002.obj
 0002:00001090       ??_C@_0BO@EOHGKJHI@JVMTI_ERROR_UNATTACHED_THREAD@ 0000000180007090     libthrcputime002.obj
 0002:000010b0       ??_C@_0CA@LKHFDACL@JVMTI_ERROR_INVALID_ENVIRONMENT@ 00000001800070b0     libthrcputime002.obj
 0002:000010d0       ??_C@_0BA@MMFHLOKK@?$DMunknown?5error?$DO@ 00000001800070d0     libthrcputime002.obj
 0002:000010e0       ??_C@_0CF@CBHOKDB@throwable?5?$DN?5jni?9?$DOExceptionOccur@ 00000001800070e0     libthrcputime002.obj
 0002:00001108       ??_C@_03OFAPEBGM@?$CFs?6@  0000000180007108     libthrcputime002.obj
 0002:00001110       ??_C@_0DM@LPIGEGNJ@s?2test?2hotspot?2jtreg?2vmTestbase@ 0000000180007110     libthrcputime002.obj
 0002:00001150       ??_C@_0CC@NFCNPEPK@Exception?5in?5JNI?5call?5?$CIcleared?$CJ@ 0000000180007150     libthrcputime002.obj
 0002:00001178       ??_C@_0BJ@IBAKFIKF@jni?9?$DOExceptionDescribe?$CI?$CJ@ 0000000180007178     libthrcputime002.obj
 0002:00001198       ??_C@_0BG@GGKALKMH@jni?9?$DOExceptionClear?$CI?$CJ@ 0000000180007198     libthrcputime002.obj
 0002:000011b0       ??_C@_0CF@JMGFGJLJ@?$CD?5?5?5verified?5JNI?5assertion?5is?5F@ 00000001800071b0     libthrcputime002.obj
 0002:000011d8       ??_C@_07KBAMPNJK@verbose@  00000001800071d8     libthrcputime002.obj
 0002:000011e0       ??_C@_0DN@PKJBOLAP@nsk_jvmti_parseOptions?$CI?$CJ?3?5unexp@ 00000001800071e0     libthrcputime002.obj
 0002:00001220       ??_C@_05IMBNNINJ@trace@    0000000180007220     libthrcputime002.obj
 0002:00001228       ??_C@_0DD@BJKGNDMB@nsk_jvmti_parseOptions?$CI?$CJ?3?5no?5va@ 0000000180007228     libthrcputime002.obj
 0002:0000125c       ??_C@_04CGFJFPFD@none@     000000018000725c     libthrcputime002.obj
 0002:00001264       ??_C@_06BMELKFMA@before@   0000000180007264     libthrcputime002.obj
 0002:0000126c       ??_C@_05CMKPCFDK@after@    000000018000726c     libthrcputime002.obj
 0002:00001274       ??_C@_03NFKEKGGK@all@      0000000180007274     libthrcputime002.obj
 0002:00001278       ??_C@_0DM@NDNJGJKE@nsk_jvmti_parseOptions?$CI?$CJ?3?5uexpe@ 0000000180007278     libthrcputime002.obj
 0002:000012b8       ??_C@_08NBBJKJO@waittime@  00000001800072b8     libthrcputime002.obj
 0002:000012c8       ??_C@_0DO@CMHGAOHC@nsk_jvmti_parseOptions?$CI?$CJ?3?5not?5i@ 00000001800072c8     libthrcputime002.obj
 0002:00001308       ??_C@_0DL@LNMPBDLN@nsk_jvmti_parseOptions?$CI?$CJ?3?5negat@ 0000000180007308     libthrcputime002.obj
 0002:00001348       ??_C@_0DA@GMFJNOJH@nsk_jvmti_parseOptions?$CI?$CJ?3?5unkno@ 0000000180007348     libthrcputime002.obj
 0002:00001378       ??_C@_0CO@CCIAMEAN@nsk_jvmti_parseOptions?$CI?$CJ?3?5found@ 0000000180007378     libthrcputime002.obj
 0002:000013a8       ??_C@_0CJ@OEGPCGDL@nsk_jvmti_parseOptions?$CI?$CJ?3?5out?5o@ 00000001800073a8     libthrcputime002.obj
 0002:000013d8       ??_C@_0DI@NMBHPGGF@nsk_jvmti_parseOptions?$CI?$CJ?3?5too?5m@ 00000001800073d8     libthrcputime002.obj
 0002:00001410       ??_C@_03POGCGECB@?5?0?$HO@ 0000000180007410     libthrcputime002.obj
 0002:00001418       ??_C@_0DC@GKLNPJIJ@nsk_jvmti_findOptionValue?$CI?$CJ?3?5op@ 0000000180007418     libthrcputime002.obj
 0002:00001450       ??_C@_0DF@OPPIHBPJ@nsk_jvmti_findOptionIntValue?$CI?$CJ?3@ 0000000180007450     libthrcputime002.obj
 0002:00001488       ??_C@_0DO@DBKDODPI@nsk_jvmti_findOptionIntValue?$CI?$CJ?3@ 0000000180007488     libthrcputime002.obj
 0002:000014d0       ??_C@_0EE@NGNPKOJC@nsk_jvmti_findOptionIntValue?$CI?$CJ?3@ 00000001800074d0     libthrcputime002.obj
 0002:00001518       ??_C@_0CB@MLNJNCLJ@?5?5jvmti?5error?3?5code?$DN?$CFd?0?5name?$DN?$CFs@ 0000000180007518     libthrcputime002.obj
 0002:00001540       ??_C@_0CD@OHBGDKMK@?$CD?5?5?5jvmti?5error?3?5code?$DN?$CFd?0?5name?$DN@ 0000000180007540     libthrcputime002.obj
 0002:00001568       ??_C@_0CG@JNNCGPHB@?$CD?5?5?5error?5expected?3?5code?$DN?$CFd?0?5na@ 0000000180007568     libthrcputime002.obj
 0002:00001590       ??_C@_0EB@IMGKPCGE@?$CIstr_obj?5?$DN?5jni?9?$DONewStringUTF?$CIco@ 0000000180007590     libthrcputime002.obj
 0002:000015e0       ??_C@_0EA@HFOGGBCC@s?2test?2hotspot?2jtreg?2vmTestbase@ 00000001800075e0     libthrcputime002.obj
 0002:00001620       ??_C@_05KKCIMGE@error@     0000000180007620     libthrcputime002.obj
 0002:00001628       ??_C@_0CJ@JACLEAA@Test?5failed?5by?5setFailStatus?$CI?$CJ?4@ 0000000180007628     libthrcputime002.obj
 0002:00001658       ??_C@_0BD@HGNAOMCP@agent_data_monitor@ 0000000180007658     libthrcputime002.obj
 0002:00001670       ??_C@_0EB@OGCLGKLN@javaVM?9?$DOGetEnv?$CI?$CIvoid?5?$CK?$CK?$CJ?$CGjvmti_@ 0000000180007670     libthrcputime002.obj
 0002:000016c0       ??_C@_0EA@PNBCDMOA@s?2test?2hotspot?2jtreg?2vmTestbase@ 00000001800076c0     libthrcputime002.obj
 0002:00001700       ??_C@_0CI@DDPIFBGM@init_agent_data?$CIjvmti_env?0?5?$CGage@ 0000000180007700     libthrcputime002.obj
 0002:00001728       ??_C@_0DI@ILAHDLMP@?$CI?$CKagentThreadProc?$CJ?$CIjvmti_env?0?5a@ 0000000180007728     libthrcputime002.obj
 0002:00001760       ??_C@_0BD@KDBALNLB@JVMTI?5agent?5thread@ 0000000180007760     libthrcputime002.obj
 0002:00001778       ??_C@_0BB@NOKBFPFO@java?1lang?1Thread@ 0000000180007778     libthrcputime002.obj
 0002:0000178c       ??_C@_06FALKBLGB@?$DMinit?$DO@ 000000018000778c     libthrcputime002.obj
 0002:00001798       ??_C@_0BG@IKDDPPGD@?$CILjava?1lang?1String?$DL?$CJV@ 0000000180007798     libthrcputime002.obj
 0002:000017b0       ??_C@_0EB@IFJBFEKC@?$CIthreadClass?5?$DN?5jni_env?9?$DOFindCla@ 00000001800077b0     libthrcputime002.obj
 0002:00001800       ??_C@_0GF@FGFIBKKL@?$CIthreadCtor?5?$DN?5jni_env?9?$DOGetMetho@ 0000000180007800     libthrcputime002.obj
 0002:00001868       ??_C@_0DN@NCPDJLOG@?$CIthreadName?5?$DN?5jni_env?9?$DONewStrin@ 0000000180007868     libthrcputime002.obj
 0002:000018b0       ??_C@_0FE@PFKODBGC@?$CIthreadObject?5?$DN?5jni_env?9?$DONewObj@ 00000001800078b0     libthrcputime002.obj
 0002:00001910       ??_C@_0ED@HOBAHHJI@?$CIthreadGlobalRef?5?$DN?5jni_env?9?$DONew@ 0000000180007910     libthrcputime002.obj
 0002:00001960       ??_C@_0FN@HNJJAHFC@jvmti_env?9?$DORunAgentThread?$CIagent@ 0000000180007960     libthrcputime002.obj
 0002:000019c0       ??_C@_0EA@MOJDNKDF@Debuggee?5status?5sync?5aborted?5be@ 00000001800079c0     libthrcputime002.obj
 0002:00001a00       ??_C@_0CO@PGPGMHBJ@No?5status?5sync?5occured?5for?5time@ 0000000180007a00     libthrcputime002.obj
 0002:00001a30       ??_C@_0CL@DOEBDPKJ@Debuggee?5was?5not?5suspended?5on?5s@ 0000000180007a30     libthrcputime002.obj
 0002:00001a60       ??_C@_0EA@EEOEJAEN@status?5?$DN?5syncDebuggeeStatus?$CIjni@ 0000000180007a60     libthrcputime002.obj
 0002:00001aa0       ??_C@_0BL@JBCFNBMB@nsk_jvmti_resetAgentData?$CI?$CJ@ 0000000180007aa0     libthrcputime002.obj
 0002:00001ac0       ??_C@_0DN@NNGECJON@jvmti_env?9?$DOSetEventNotification@ 0000000180007ac0     libthrcputime002.obj
 0002:00001b00       ??_C@_0EL@LPBEELIP@s?2test?2hotspot?2jtreg?2vmTestbase@ 0000000180007b00     libthrcputime002.obj
 0002:00001b50       ??_C@_0CK@JDAMFDMJ@jvmti?9?$DOSetTag?$CIo?0?5tag?$CJ?5?$DN?$DN?5JVMTI_@ 0000000180007b50     libthrcputime002.obj
 0002:00001b80       ??_C@_0CC@DAMNHKNI@Can?8t?5set?5tag?5?$CFli?5for?5object?5?$CFl@ 0000000180007b80     libthrcputime002.obj
 0002:00001ba8       ??_C@_0DL@HAJPNKEF@jvmti?9?$DOGetObjectHashCode?$CIo?0?5?$CGha@ 0000000180007ba8     libthrcputime002.obj
 0002:00001be8       ??_C@_0BL@JFPIEOBF@Can?8t?5get?5hash?5object?5?$CFlx?6@ 0000000180007be8     libthrcputime002.obj
 0002:00001c08       ??_C@_0BG@DICPHBKN@setTag?3?5?$CF08x?5?$DM?9?5?$CF?53li@ 0000000180007c08     libthrcputime002.obj
 0002:00001c20       ??_C@_0DH@FCEEBDMJ@?$CIs?5?$DN?5jni?9?$DOGetStringUTFChars?$CIsIn@ 0000000180007c20     libthrcputime002.obj
 0002:00001c58       ??_C@_0BJ@OKKGHDCN@Can?8t?5get?5string?5at?5?$CF?$CDp?6@ 0000000180007c58     libthrcputime002.obj
 0002:00001c78       ??_C@_0BP@EKFLGGFJ@Can?8t?5get?5string?5at?5?$CF?$CDp?3?5null?6@ 0000000180007c78     libthrcputime002.obj
 0002:00001c98       ??_C@_06ICODBHCL@?5?1?1?5?$CFs@ 0000000180007c98     libthrcputime002.obj
 0002:00001ca0       ??_C@_0DB@KGFPLEGO@?$CIr?5?$DN?5jvmti?9?$DOGetTag?$CIo?0?5?$CGtag?$CJ?$CJ?5?$DN?$DN@ 0000000180007ca0     libthrcputime002.obj
 0002:00001cd8       ??_C@_0CO@PDAGBCGJ@Can?8t?5GetTag?5for?5object?5?$CFlx?4?5Re@ 0000000180007cd8     libthrcputime002.obj
 0002:00001d08       ??_C@_0CH@HPEODOHC@TEST_BUG?3?5Max?4?5number?5of?5refs?5r@ 0000000180007d08     libthrcputime002.obj
 0002:00001d30       ??_C@_0DI@PHFCABIM@?$CIr?5?$DN?5jvmti?9?$DOGetTag?$CIfrom?0?5?$CGtagFr@ 0000000180007d30     libthrcputime002.obj
 0002:00001d68       ??_C@_0DI@MDEGFNKD@TEST_BUG?3?5Can?8t?5GetTag?5for?5obje@ 0000000180007d68     libthrcputime002.obj
 0002:00001da0       ??_C@_0DE@MLELJAHM@?$CIr?5?$DN?5jvmti?9?$DOGetTag?$CIto?0?5?$CGtagTo?$CJ?$CJ@ 0000000180007da0     libthrcputime002.obj
 0002:00001dd8       ??_C@_0CF@LHDNIPGP@GetThreadCpuTime?$CI?$CJ?5for?5thread?3?5@ 0000000180007dd8     libthrcputime002.obj
 0002:00001e00       ??_C@_0FL@FJFEPNBM@s?2test?2hotspot?2jtreg?2vmTestbase@ 0000000180007e00     libthrcputime002.obj
 0002:00001e60       ??_C@_0CP@IMANAKFF@jvmti?9?$DOGetThreadCpuTime?$CIthread?0@ 0000000180007e60     libthrcputime002.obj
 0002:00001e90       ??_C@_0BI@BMALLB@?5?5?4?4?4?5got?5cpu?5time?3?5?$CFs?6@ 0000000180007e90     libthrcputime002.obj
 0002:00001eb0       ??_C@_0EA@CMPOALHE@?$CD?5WARNING?3?5In?5?$CFs?5GetThreadCpuTi@ 0000000180007eb0     libthrcputime002.obj
 0002:00001ef0       ??_C@_0CA@NGIPCDBE@Compare?5with?5previous?5time?3?5?$CFs?6@ 0000000180007ef0     libthrcputime002.obj
 0002:00001f10       ??_C@_0BG@PNCPIDEL@?5?5?4?4?4?5difference?3?5?$CFs?6@ 0000000180007f10     libthrcputime002.obj
 0002:00001f30       ??_C@_0HG@DEHBLNAA@In?5?$CFs?5GetThreadCpuTime?$CI?$CJ?5return@ 0000000180007f30     libthrcputime002.obj
 0002:00001fb0       ??_C@_0HA@DGOIFEPA@?$CD?5WARNING?3?5In?5?$CFs?5GetThreadCpuTi@ 0000000180007fb0     libthrcputime002.obj
 0002:00002020       ??_C@_0BM@BJPDIKEG@Started?5agent?5thread?3?50x?$CFp?6@ 0000000180008020     libthrcputime002.obj
 0002:00002040       ??_C@_0CC@HCPFMLEK@Wait?5for?5debugee?5to?5become?5read@ 0000000180008040     libthrcputime002.obj
 0002:00002068       ??_C@_0DJ@MFPBEABO@?$DO?$DO?$DO?5Testcase?5?$CD2?3?5Check?5initial?5@ 0000000180008068     libthrcputime002.obj
 0002:000020a8       ??_C@_0N@POFOADDC@agent?5thread@ 00000001800080a8     libthrcputime002.obj
 0002:000020c0       ??_C@_0EB@MCCPONCO@?$DO?$DO?$DO?5Testcases?5?$CD3?94?07?98?3?5Check?5c@ 00000001800080c0     libthrcputime002.obj
 0002:00002108       ??_C@_0CB@ONKMCBCK@Enable?5thread?5events?3?5?$CFd?5events@ 0000000180008108     libthrcputime002.obj
 0002:00002130       ??_C@_0P@BAMBNLJF@?5?5?4?4?4?5enabled?6@ 0000000180008130     libthrcputime002.obj
 0002:00002140       ??_C@_0BM@JDGAKOHG@Let?5tested?5thread?5to?5start?6@ 0000000180008140     libthrcputime002.obj
 0002:00002160       ??_C@_0DK@NFHMGGDF@?$DO?$DO?$DO?5Testcase?5?$CD5?3?5Check?5middle?5c@ 0000000180008160     libthrcputime002.obj
 0002:000021a0       ??_C@_0EB@HGKGKNEH@?$DO?$DO?$DO?5Testcase?5?$CD6?3?5Check?5tested?5t@ 00000001800081a0     libthrcputime002.obj
 0002:000021e8       ??_C@_0BN@EBKKKNNN@Let?5tested?5thread?5to?5finish?6@ 00000001800081e8     libthrcputime002.obj
 0002:00002208       ??_C@_0CC@HDKFNDNE@Disable?5thread?5events?3?5?$CFd?5event@ 0000000180008208     libthrcputime002.obj
 0002:00002230       ??_C@_0BA@DDKAOGOI@?5?5?4?4?4?5disabled?6@ 0000000180008230     libthrcputime002.obj
 0002:00002240       ??_C@_0DH@ICBCNFAN@?$DO?$DO?$DO?5Testcase?5?$CD9?3?5Check?5final?5cp@ 0000000180008240     libthrcputime002.obj
 0002:00002278       ??_C@_0BH@HPEOJMHL@Let?5debugee?5to?5finish?6@ 0000000180008278     libthrcputime002.obj
 0002:00002290       ??_C@_0DN@GLAJFBGP@?$DO?$DO?$DO?5Testcase?5?$CD1?3?5Check?5initial?5@ 0000000180008290     libthrcputime002.obj
 0002:000022d0       ??_C@_0BB@ECBNOENI@VM_INIT?5callback@ 00000001800082d0     libthrcputime002.obj
 0002:000022e8       ??_C@_0BL@OGOOPPCN@Disable?5events?3?5?$CFd?5events?6@ 00000001800082e8     libthrcputime002.obj
 0002:00002308       ??_C@_0CA@LDMJDFDO@Exit?5with?5FAIL?5exit?5status?3?5?$CFd?6@ 0000000180008308     libthrcputime002.obj
 0002:00002328       ??_C@_0BC@PCOLJFHD@exit?$CISTATUS_FAIL?$CJ@ 0000000180008328     libthrcputime002.obj
 0002:00002340       ??_C@_0CK@NPKDGJFI@jvmti?9?$DOGetThreadInfo?$CIthread?0?5?$CGt@ 0000000180008340     libthrcputime002.obj
 0002:00002370       ??_C@_0CD@IOGKHOKH@?5?5?5?5?$DMTHREAD_START?$DO?5for?5thread?3?5@ 0000000180008370     libthrcputime002.obj
 0002:000023a0       ??_C@_0EH@FEJMBNGG@?$DO?$DO?$DO?5Testcase?5?$CD3?3?5Check?5agent?5th@ 00000001800083a0     libthrcputime002.obj
 0002:000023e8       ??_C@_0BG@JINAKLHL@THREAD_START?5callback@ 00000001800083e8     libthrcputime002.obj
 0002:00002400       ??_C@_0BE@INPECBPC@thrcputime002Thread@ 0000000180008400     libthrcputime002.obj
 0002:00002418       ??_C@_0DG@IFONIIMN@?$CItestedThread?5?$DN?5jni?9?$DONewGlobalR@ 0000000180008418     libthrcputime002.obj
 0002:00002450       ??_C@_0EC@JPABONKK@?$DO?$DO?$DO?5Testcase?5?$CD4?3?5Check?5initial?5@ 0000000180008450     libthrcputime002.obj
 0002:00002498       ??_C@_0CD@ILAPIHMG@?5?5?5?5?$DMTHREAD_END?$DO?5?5?5for?5thread?3?5@ 0000000180008498     libthrcputime002.obj
 0002:000024c0       ??_C@_0EF@LMMDKPEC@?$DO?$DO?$DO?5Testcase?5?$CD7?3?5Check?5agent?5th@ 00000001800084c0     libthrcputime002.obj
 0002:00002508       ??_C@_0BE@BAAPBFGJ@THREAD_END?5callback@ 0000000180008508     libthrcputime002.obj
 0002:00002520       ??_C@_0DO@CPNKMHAJ@?$DO?$DO?$DO?5Testcase?5?$CD8?3?5Check?5final?5cp@ 0000000180008520     libthrcputime002.obj
 0002:00002560       ??_C@_0CD@JEIIOPBJ@jni?9?$DODeleteGlobalRef?$CItestedThre@ 0000000180008560     libthrcputime002.obj
 0002:00002588       ??_C@_0CA@MNKGCBCG@nsk_jvmti_parseOptions?$CIoptions?$CJ@ 0000000180008588     libthrcputime002.obj
 0002:000025a8       ??_C@_0L@LEIMKHLK@iterations@ 00000001800085a8     libthrcputime002.obj
 0002:000025b8       ??_C@_0BD@COGOFEE@iterations?5?$DO?$DN?51000@ 00000001800085b8     libthrcputime002.obj
 0002:000025d0       ??_C@_0DN@MIAMNFPH@?$CIjvmti?5?$DN?5nsk_jvmti_createJVMTIE@ 00000001800085d0     libthrcputime002.obj
 0002:00002610       ??_C@_0BI@PCABJHOG@can_get_thread_cpu_time@ 0000000180008610     libthrcputime002.obj
 0002:00002628       ??_C@_0BN@MBBGLOKH@Add?5required?5capability?3?5?$CFs?6@ 0000000180008628     libthrcputime002.obj
 0002:00002648       ??_C@_0BO@DBKDIPGD@jvmti?9?$DOAddCapabilities?$CI?$CGcaps?$CJ@ 0000000180008648     libthrcputime002.obj
 0002:00002668       ??_C@_0BI@IMBFLOOI@?5?5?4?4?4?5capability?5added?6@ 0000000180008668     libthrcputime002.obj
 0002:00002680       ??_C@_0CM@EOIMPJOL@VM_INIT?0?5VM_DEATH?0?5THREAD_START@ 0000000180008680     libthrcputime002.obj
 0002:000026b0       ??_C@_0BK@DMBLKMAE@Set?5events?5callbacks?3?5?$CFs?6@ 00000001800086b0     libthrcputime002.obj
 0002:000026d0       ??_C@_0EC@ODFGFOAJ@jvmti?9?$DOSetEventCallbacks?$CI?$CGevent@ 00000001800086d0     libthrcputime002.obj
 0002:00002718       ??_C@_0BF@FJCGAMPH@?5?5?4?4?4?5callbacks?5set?6@ 0000000180008718     libthrcputime002.obj
 0002:00002730       ??_C@_0CL@PIACJIPK@nsk_jvmti_setAgentProc?$CIagentPro@ 0000000180008730     libthrcputime002.obj
 0002:00002760       ??_C@_0BK@EKNILGAD@Enable?5events?3?5?$CFd?5events?6@ 0000000180008760     libthrcputime002.obj
 0002:00002780       ??_C@_0CA@NCMBDOKI@Raw?5monitor?5for?5synchronization@ 0000000180008780     libthrcputime002.obj
 0002:000027b0       ??_C@_1EC@JIJBPKFM@?$AAa?$AAp?$AAi?$AA?9?$AAm?$AAs?$AA?9?$AAw?$AAi?$AAn?$AA?9?$AAc?$AAo?$AAr?$AAe@ 00000001800087b0     MSVCRT:thread_safe_statics.obj
 0002:000027f8       ??_C@_1BK@MGMFAEKH@?$AAk?$AAe?$AAr?$AAn?$AAe?$AAl?$AA3?$AA2?$AA?4?$AAd?$AAl?$AAl@ 00000001800087f8     MSVCRT:thread_safe_statics.obj
 0002:00002818       ??_C@_0BJ@JEBJOJFJ@SleepConditionVariableCS@ 0000000180008818     MSVCRT:thread_safe_statics.obj
 0002:00002838       ??_C@_0BJ@PGPPEPCC@WakeAllConditionVariable@ 0000000180008838     MSVCRT:thread_safe_statics.obj
 0002:00002858       _pDefaultRawDllMain        0000000180008858     MSVCRT:dll_dllmain.obj
 0002:00002858       _pRawDllMain               0000000180008858     MSVCRT:dll_dllmain.obj
 0002:00002860       __xmm@ffffffffffffffffffffffffffffffff 0000000180008860     MSVCRT:utility.obj
 0002:00002870       _load_config_used          0000000180008870     MSVCRT:loadcfg.obj
 0002:00002a80       _tls_used                  0000000180008a80     MSVCRT:tlssup.obj
 0002:00002aa8       __volatile_metadata        0000000180008aa8     <linker-defined>
 0002:00002e80       __rtc_iaa                  0000000180008e80     MSVCRT:initsect.obj
 0002:00002e88       __rtc_izz                  0000000180008e88     MSVCRT:initsect.obj
 0002:00002e90       __rtc_taa                  0000000180008e90     MSVCRT:initsect.obj
 0002:00002e98       __rtc_tzz                  0000000180008e98     MSVCRT:initsect.obj
 0002:00002ea0       _tls_start                 0000000180008ea0     MSVCRT:tlssup.obj
 0002:00002ea4       _Init_thread_epoch         0000000180008ea4     MSVCRT:thread_safe_statics.obj
 0002:00002ea8       _tls_end                   0000000180008ea8     MSVCRT:tlssup.obj
 0002:00003674       __IMPORT_DESCRIPTOR_KERNEL32 0000000180009674     kernel32:KERNEL32.dll
 0002:00003688       __IMPORT_DESCRIPTOR_VCRUNTIME140 0000000180009688     vcruntime:VCRUNTIME140.dll
 0002:0000369c       __IMPORT_DESCRIPTOR_api-ms-win-crt-heap-l1-1-0 000000018000969c     ucrt:api-ms-win-crt-heap-l1-1-0.dll
 0002:000036b0       __IMPORT_DESCRIPTOR_api-ms-win-crt-runtime-l1-1-0 00000001800096b0     ucrt:api-ms-win-crt-runtime-l1-1-0.dll
 0002:000036c4       __IMPORT_DESCRIPTOR_api-ms-win-crt-convert-l1-1-0 00000001800096c4     ucrt:api-ms-win-crt-convert-l1-1-0.dll
 0002:000036d8       __IMPORT_DESCRIPTOR_api-ms-win-crt-stdio-l1-1-0 00000001800096d8     ucrt:api-ms-win-crt-stdio-l1-1-0.dll
 0002:000036ec       __IMPORT_DESCRIPTOR_api-ms-win-crt-string-l1-1-0 00000001800096ec     ucrt:api-ms-win-crt-string-l1-1-0.dll
 0002:00003700       __NULL_IMPORT_DESCRIPTOR   0000000180009700     kernel32:KERNEL32.dll
 0003:00000040       _Init_global_epoch         000000018000a040     MSVCRT:thread_safe_statics.obj
 0003:00000050       __security_cookie          000000018000a050     MSVCRT:gs_cookie.obj
 0003:00000058       __security_cookie_complement 000000018000a058     MSVCRT:gs_cookie.obj
 0003:00000060       __scrt_native_dllmain_reason 000000018000a060     MSVCRT:utility.obj
 0003:00000068       __isa_available            000000018000a068     MSVCRT:cpu_disp.obj
 0003:0000006c       __isa_enabled              000000018000a06c     MSVCRT:cpu_disp.obj
 0003:00000070       __memset_fast_string_threshold 000000018000a070     MSVCRT:cpu_disp.obj
 0003:00000078       __memset_nt_threshold      000000018000a078     MSVCRT:cpu_disp.obj
 0003:00000080       __scrt_ucrt_dll_is_in_use  000000018000a080     MSVCRT:ucrt_stubs.obj
 0003:00000090       g_wrongHeapCallbacks       000000018000a090     libthrcputime002.obj
 0003:00000110       g_szTagInfo                000000018000a110     libthrcputime002.obj
 0003:00002050       g_tagFlags                 000000018000c050     libthrcputime002.obj
 0003:00002438       g_refsToVerifyCnt          000000018000c438     libthrcputime002.obj
 0003:0000243c       g_fakeUserData             000000018000c43c     libthrcputime002.obj
 0003:00002440       g_tagVisitCount            000000018000c440     libthrcputime002.obj
 0003:000033e0       g_refsToVerify             000000018000d3e0     libthrcputime002.obj
 0003:0001aae0       g_userDataError            0000000180024ae0     libthrcputime002.obj
 0003:0001aca8       ?_OptionsStorage@?1??__local_stdio_printf_options@@9@4_KA 0000000180024ca8     libthrcputime002.obj
 0003:0001b268       _tls_index                 0000000180025268     MSVCRT:tlssup.obj
 0003:0001b270       __scrt_current_native_startup_state 0000000180025270     MSVCRT:utility.obj
 0003:0001b278       __scrt_native_startup_lock 0000000180025278     MSVCRT:utility.obj
 0003:0001b2b8       __scrt_debugger_hook_flag  00000001800252b8     MSVCRT:utility_desktop.obj
 0003:0001b2c0       ?__type_info_root_node@@3U__type_info_node@@A 00000001800252c0     MSVCRT:tncleanup.obj
 0003:0001b2d0       ?_OptionsStorage@?1??__local_stdio_scanf_options@@9@4_KA 00000001800252d0     MSVCRT:default_local_stdio_options.obj
 0003:0001b2d8       __favor                    00000001800252d8     MSVCRT:cpu_disp.obj
 0003:0001b2e0       __dyn_tls_init_callback    00000001800252e0     <common>

 entry point at        0001:00003a90

 Static symbols

 0000:fffd8000       .debug$S                   0000000180000000     thrcputime002.exp
 0000:fffd8000       .debug$S                   0000000180000000     vcruntime:VCRUNTIME140.dll
 0000:fffd8000       .debug$S                   0000000180000000     vcruntime:VCRUNTIME140.dll
 0000:fffd8000       .debug$S                   0000000180000000     vcruntime:VCRUNTIME140.dll
 0000:fffd8000       .debug$S                   0000000180000000     vcruntime:VCRUNTIME140.dll
 0000:fffd8000       .debug$S                   0000000180000000     vcruntime:VCRUNTIME140.dll
 0000:fffd8000       .debug$S                   0000000180000000     vcruntime:VCRUNTIME140.dll
 0000:fffd8000       .debug$S                   0000000180000000     vcruntime:VCRUNTIME140.dll
 0000:fffd8000       .debug$S                   0000000180000000     ucrt:api-ms-win-crt-convert-l1-1-0.dll
 0000:fffd8000       .debug$S                   0000000180000000     ucrt:api-ms-win-crt-heap-l1-1-0.dll
 0000:fffd8000       .debug$S                   0000000180000000     ucrt:api-ms-win-crt-heap-l1-1-0.dll
 0000:fffd8000       .debug$S                   0000000180000000     ucrt:api-ms-win-crt-heap-l1-1-0.dll
 0000:fffd8000       .debug$S                   0000000180000000     ucrt:api-ms-win-crt-heap-l1-1-0.dll
 0000:fffd8000       .debug$S                   0000000180000000     ucrt:api-ms-win-crt-runtime-l1-1-0.dll
 0000:fffd8000       .debug$S                   0000000180000000     ucrt:api-ms-win-crt-runtime-l1-1-0.dll
 0000:fffd8000       .debug$S                   0000000180000000     ucrt:api-ms-win-crt-runtime-l1-1-0.dll
 0000:fffd8000       .debug$S                   0000000180000000     ucrt:api-ms-win-crt-runtime-l1-1-0.dll
 0000:fffd8000       .debug$S                   0000000180000000     ucrt:api-ms-win-crt-runtime-l1-1-0.dll
 0000:fffd8000       .debug$S                   0000000180000000     ucrt:api-ms-win-crt-runtime-l1-1-0.dll
 0000:fffd8000       .debug$S                   0000000180000000     ucrt:api-ms-win-crt-runtime-l1-1-0.dll
 0000:fffd8000       .debug$S                   0000000180000000     ucrt:api-ms-win-crt-runtime-l1-1-0.dll
 0000:fffd8000       .debug$S                   0000000180000000     ucrt:api-ms-win-crt-runtime-l1-1-0.dll
 0000:fffd8000       .debug$S                   0000000180000000     ucrt:api-ms-win-crt-runtime-l1-1-0.dll
 0000:fffd8000       .debug$S                   0000000180000000     ucrt:api-ms-win-crt-runtime-l1-1-0.dll
 0000:fffd8000       .debug$S                   0000000180000000     ucrt:api-ms-win-crt-runtime-l1-1-0.dll
 0000:fffd8000       .debug$S                   0000000180000000     ucrt:api-ms-win-crt-runtime-l1-1-0.dll
 0000:fffd8000       .debug$S                   0000000180000000     ucrt:api-ms-win-crt-runtime-l1-1-0.dll
 0000:fffd8000       .debug$S                   0000000180000000     ucrt:api-ms-win-crt-runtime-l1-1-0.dll
 0000:fffd8000       .debug$S                   0000000180000000     ucrt:api-ms-win-crt-runtime-l1-1-0.dll
 0000:fffd8000       .debug$S                   0000000180000000     ucrt:api-ms-win-crt-stdio-l1-1-0.dll
 0000:fffd8000       .debug$S                   0000000180000000     ucrt:api-ms-win-crt-stdio-l1-1-0.dll
 0000:fffd8000       .debug$S                   0000000180000000     ucrt:api-ms-win-crt-stdio-l1-1-0.dll
 0000:fffd8000       .debug$S                   0000000180000000     ucrt:api-ms-win-crt-stdio-l1-1-0.dll
 0000:fffd8000       .debug$S                   0000000180000000     ucrt:api-ms-win-crt-stdio-l1-1-0.dll
 0000:fffd8000       .debug$S                   0000000180000000     ucrt:api-ms-win-crt-stdio-l1-1-0.dll
 0000:fffd8000       .debug$S                   0000000180000000     ucrt:api-ms-win-crt-stdio-l1-1-0.dll
 0000:fffd8000       .debug$S                   0000000180000000     ucrt:api-ms-win-crt-stdio-l1-1-0.dll
 0000:fffd8000       .debug$S                   0000000180000000     ucrt:api-ms-win-crt-stdio-l1-1-0.dll
 0000:fffd8000       .debug$S                   0000000180000000     ucrt:api-ms-win-crt-stdio-l1-1-0.dll
 0000:fffd8000       .debug$S                   0000000180000000     ucrt:api-ms-win-crt-string-l1-1-0.dll
 0000:fffd8000       .debug$S                   0000000180000000     ucrt:api-ms-win-crt-string-l1-1-0.dll
 0000:fffd8000       .debug$S                   0000000180000000     ucrt:api-ms-win-crt-string-l1-1-0.dll
 0000:fffd8000       .debug$S                   0000000180000000     ucrt:api-ms-win-crt-string-l1-1-0.dll
 0000:fffd8000       .debug$S                   0000000180000000     ucrt:api-ms-win-crt-string-l1-1-0.dll
 0000:fffd8000       .debug$S                   0000000180000000     ucrt:api-ms-win-crt-string-l1-1-0.dll
 0000:fffd8000       .debug$S                   0000000180000000     ucrt:api-ms-win-crt-string-l1-1-0.dll
 0000:fffd8000       .debug$S                   0000000180000000     ucrt:api-ms-win-crt-string-l1-1-0.dll
 0000:fffd8000       .debug$S                   0000000180000000     kernel32:KERNEL32.dll
 0000:fffd8000       .debug$S                   0000000180000000     kernel32:KERNEL32.dll
 0000:fffd8000       .debug$S                   0000000180000000     kernel32:KERNEL32.dll
 0000:fffd8000       .debug$S                   0000000180000000     kernel32:KERNEL32.dll
 0000:fffd8000       .debug$S                   0000000180000000     kernel32:KERNEL32.dll
 0000:fffd8000       .debug$S                   0000000180000000     kernel32:KERNEL32.dll
 0000:fffd8000       .debug$S                   0000000180000000     kernel32:KERNEL32.dll
 0000:fffd8000       .debug$S                   0000000180000000     kernel32:KERNEL32.dll
 0000:fffd8000       .debug$S                   0000000180000000     kernel32:KERNEL32.dll
 0000:fffd8000       .debug$S                   0000000180000000     kernel32:KERNEL32.dll
 0000:fffd8000       .debug$S                   0000000180000000     kernel32:KERNEL32.dll
 0000:fffd8000       .debug$S                   0000000180000000     kernel32:KERNEL32.dll
 0000:fffd8000       .debug$S                   0000000180000000     kernel32:KERNEL32.dll
 0000:fffd8000       .debug$S                   0000000180000000     kernel32:KERNEL32.dll
 0000:fffd8000       .debug$S                   0000000180000000     kernel32:KERNEL32.dll
 0000:fffd8000       .debug$S                   0000000180000000     kernel32:KERNEL32.dll
 0000:fffd8000       .debug$S                   0000000180000000     kernel32:KERNEL32.dll
 0000:fffd8000       .debug$S                   0000000180000000     kernel32:KERNEL32.dll
 0000:fffd8000       .debug$S                   0000000180000000     kernel32:KERNEL32.dll
 0000:fffd8000       .debug$S                   0000000180000000     kernel32:KERNEL32.dll
 0000:fffd8000       .debug$S                   0000000180000000     kernel32:KERNEL32.dll
 0000:fffd8000       .debug$S                   0000000180000000     kernel32:KERNEL32.dll
 0000:fffd8000       .debug$S                   0000000180000000     kernel32:KERNEL32.dll
 0000:fffd8000       .debug$S                   0000000180000000     kernel32:KERNEL32.dll
 0000:fffd8000       .debug$S                   0000000180000000     kernel32:KERNEL32.dll
 0000:fffd8000       .debug$S                   0000000180000000     kernel32:KERNEL32.dll
 0000:fffd8000       .debug$S                   0000000180000000     kernel32:KERNEL32.dll
 0000:fffd8000       .debug$S                   0000000180000000     kernel32:KERNEL32.dll
 0001:000002ec       ?check_jvmti_status@@YAXPEAUJNIEnv_@@W4jvmtiError@@PEBD@Z 00000001800012ec f   libthrcputime002.obj
 0001:00001148       addRefToVerify             0000000180002148 f   libthrcputime002.obj
 0001:000011b4       agentProc                  00000001800021b4 f   libthrcputime002.obj
 0001:00001568       agentThreadWrapper         0000000180002568 f   libthrcputime002.obj
 0001:00001d2c       checkCpuTime               0000000180002d2c f   libthrcputime002.obj
 0001:00001f80       check_option               0000000180002f80 f   libthrcputime002.obj
 0001:000021c8       file_basename              00000001800031c8 f   libthrcputime002.obj
 0001:00002f74       startAgentThreadWrapper    0000000180003f74 f   libthrcputime002.obj
 0001:000032b4       syncDebuggeeStatus         00000001800042b4 f   libthrcputime002.obj
 0001:00003554       capture_previous_context   0000000180004554 f   MSVCRT:gs_report.obj
 0001:000035c8       ?__scrt_initialize_thread_safe_statics@@YAHXZ 00000001800045c8 f   MSVCRT:thread_safe_statics.obj
 0001:00003698       ?__scrt_uninitialize_thread_safe_statics@@YAXXZ 0000000180004698 f   MSVCRT:thread_safe_statics.obj
 0001:00003740       $$000000                   0000000180004740     MSVCRT:amdsecgs.obj
 0001:00003770       ?dllmain_crt_dispatch@@YAHQEAUHINSTANCE__@@KQEAX@Z 0000000180004770 f   MSVCRT:dll_dllmain.obj
 0001:000037c0       ?dllmain_crt_process_attach@@YAHQEAUHINSTANCE__@@QEAX@Z 00000001800047c0 f   MSVCRT:dll_dllmain.obj
 0001:000038d8       ?dllmain_crt_process_detach@@YAH_N@Z 00000001800048d8 f   MSVCRT:dll_dllmain.obj
 0001:0000395c       ?dllmain_dispatch@@YAHQEAUHINSTANCE__@@KQEAX@Z 000000018000495c f   MSVCRT:dll_dllmain.obj
 0001:00004370       $$000000                   0000000180005370     MSVCRT:guard_dispatch.obj
 0001:00004390       $$000000                   0000000180005390     MSVCRT:guard_xfg_dispatch.obj
 0001:000043a6       ?fin$0@?0??dllmain_crt_process_attach@@YAHQEAUHINSTANCE__@@QEAX@Z@4HA 00000001800053a6 f   MSVCRT:dll_dllmain.obj
 0001:000043bd       ?fin$0@?0??dllmain_crt_process_detach@@YAH_N@Z@4HA 00000001800053bd f   MSVCRT:dll_dllmain.obj
 0001:000043d6       ?fin$1@?0??dllmain_crt_process_detach@@YAH_N@Z@4HA 00000001800053d6 f   MSVCRT:dll_dllmain.obj
 0001:000043ea       ?filt$0@?0??dllmain_dispatch@@YAHQEAUHINSTANCE__@@KQEAX@Z@4HA 00000001800053ea f   MSVCRT:dll_dllmain.obj
 0001:00004420       __scrt_is_nonwritable_in_current_image$filt$0 0000000180005420 f   MSVCRT:utility.obj
 0002:00000218       ?__scrt_initialize_tss_var@@3P6AHXZEA 0000000180006218     MSVCRT:thread_safe_statics.obj
 0002:00000340       ?opcLengths@@3QBEB         0000000180006340     libthrcputime002.obj
 0002:000027a0       GS_ExceptionPointers       00000001800087a0     MSVCRT:gs_report.obj
 0002:00002eb0       $unwind$fprintf            0000000180008eb0     libthrcputime002.obj
 0002:00002ebc       $unwind$printf             0000000180008ebc     libthrcputime002.obj
 0002:00002ec8       $unwind$?NewObject@JNIEnv_@@QEAAPEAV_jobject@@PEAV_jclass@@PEAU_jmethodID@@ZZ 0000000180008ec8     libthrcputime002.obj
 0002:00002ec8       $unwind$nsk_lcomplain      0000000180008ec8     libthrcputime002.obj
 0002:00002ec8       $unwind$nsk_ldisplay       0000000180008ec8     libthrcputime002.obj
 0002:00002ed0       $unwind$nsk_jvmti_waitForSync 0000000180008ed0     libthrcputime002.obj
 0002:00002ed0       $unwind$nsk_lvdisplay      0000000180008ed0     libthrcputime002.obj
 0002:00002ed0       $unwind$_RTC_Initialize    0000000180008ed0     MSVCRT:initsect.obj
 0002:00002ed0       $unwind$_RTC_Terminate     0000000180008ed0     MSVCRT:initsect.obj
 0002:00002ed0       $unwind$?__scrt_initialize_thread_safe_statics@@YAHXZ 0000000180008ed0     MSVCRT:thread_safe_statics.obj
 0002:00002edc       $unwind$nsk_complain       0000000180008edc     libthrcputime002.obj
 0002:00002edc       $unwind$nsk_printf         0000000180008edc     libthrcputime002.obj
 0002:00002ee4       $unwind$nsk_lvcomplain     0000000180008ee4     libthrcputime002.obj
 0002:00002efc       $unwind$nsk_ltrace         0000000180008efc     libthrcputime002.obj
 0002:00002efc       $unwind$__report_gsfailure 0000000180008efc     MSVCRT:gs_report.obj
 0002:00002f04       $unwind$nsk_lvtrace        0000000180008f04     libthrcputime002.obj
 0002:00002f04       $unwind$__raise_securityfailure 0000000180008f04     MSVCRT:gs_report.obj
 0002:00002f04       $unwind$__scrt_initialize_crt 0000000180008f04     MSVCRT:utility.obj
 0002:00002f04       $unwind$__scrt_initialize_onexit_tables 0000000180008f04     MSVCRT:utility.obj
 0002:00002f04       $unwind$__scrt_release_startup_lock 0000000180008f04     MSVCRT:utility.obj
 0002:00002f04       $unwind$__scrt_uninitialize_crt 0000000180008f04     MSVCRT:utility.obj
 0002:00002f04       $unwind$_onexit            0000000180008f04     MSVCRT:utility.obj
 0002:00002f0c       $unwind$nsk_lverify        0000000180008f0c     libthrcputime002.obj
 0002:00002f1c       $unwind$callbackVMDeath    0000000180008f1c     libthrcputime002.obj
 0002:00002f1c       $unwind$nsk_vprintf        0000000180008f1c     libthrcputime002.obj
 0002:00002f2c       $unwind$?julong_to_string@@YAPEAD_KPEAD@Z 0000000180008f2c     libthrcputime002.obj
 0002:00002f3c       $unwind$?check_jvmti_status@@YAXPEAUJNIEnv_@@W4jvmtiError@@PEBD@Z 0000000180008f3c     libthrcputime002.obj
 0002:00002f4c       $unwind$?create_raw_monitor@@YAPEAU_jrawMonitorID@@PEAU_jvmtiEnv@@PEBD@Z 0000000180008f4c     libthrcputime002.obj
 0002:00002f4c       $unwind$Java_nsk_jvmti_unit_FollowReferences_FollowRefObjects_resetTags 0000000180008f4c     libthrcputime002.obj
 0002:00002f4c       $unwind$addRefToVerify     0000000180008f4c     libthrcputime002.obj
 0002:00002f4c       $unwind$nsk_jvmti_resetAgentData 0000000180008f4c     libthrcputime002.obj
 0002:00002f4c       $unwind$nsk_jvmti_resumeSync 0000000180008f4c     libthrcputime002.obj
 0002:00002f4c       $unwind$nsk_jvmti_setFailStatus 0000000180008f4c     libthrcputime002.obj
 0002:00002f4c       $unwind$__scrt_initialize_default_local_stdio_options 0000000180008f4c     MSVCRT:default_local_stdio_options.obj
 0002:00002f4c       $unwind$?dllmain_crt_dispatch@@YAHQEAUHINSTANCE__@@KQEAX@Z 0000000180008f4c     MSVCRT:dll_dllmain.obj
 0002:00002f4c       $unwind$DllMain            0000000180008f4c     MSVCRT:dll_dllmain_stub.obj
 0002:00002f4c       $unwind$__GSHandlerCheck   0000000180008f4c     MSVCRT:gshandler.obj
 0002:00002f4c       $unwind$?__scrt_uninitialize_thread_safe_statics@@YAXXZ 0000000180008f4c     MSVCRT:thread_safe_statics.obj
 0002:00002f4c       $unwind$__scrt_acquire_startup_lock 0000000180008f4c     MSVCRT:utility.obj
 0002:00002f4c       $unwind$__scrt_dllmain_after_initialize_c 0000000180008f4c     MSVCRT:utility.obj
 0002:00002f4c       $unwind$__scrt_dllmain_before_initialize_c 0000000180008f4c     MSVCRT:utility.obj
 0002:00002f4c       $unwind$__scrt_dllmain_crt_thread_attach 0000000180008f4c     MSVCRT:utility.obj
 0002:00002f4c       $unwind$__scrt_dllmain_crt_thread_detach 0000000180008f4c     MSVCRT:utility.obj
 0002:00002f4c       $unwind$__scrt_dllmain_uninitialize_c 0000000180008f4c     MSVCRT:utility.obj
 0002:00002f4c       $unwind$__scrt_dllmain_uninitialize_critical 0000000180008f4c     MSVCRT:utility.obj
 0002:00002f4c       $unwind$atexit             0000000180008f4c     MSVCRT:utility.obj
 0002:00002f54       $unwind$?nsk_jni_lverify@@YAHHPEAUJNIEnv_@@HQEBDH1ZZ 0000000180008f54     libthrcputime002.obj
 0002:00002f68       $unwind$?nsk_jni_check_exception@@YAHPEAUJNIEnv_@@QEBDH@Z 0000000180008f68     libthrcputime002.obj
 0002:00002f84       $unwind$nsk_jvmti_parseOptions 0000000180008f84     libthrcputime002.obj
 0002:00002fa0       $unwind$nsk_jvmti_createJVMTIEnv 0000000180008fa0     libthrcputime002.obj
 0002:00002fb4       $unwind$nsk_jvmti_enableEvents 0000000180008fb4     libthrcputime002.obj
 0002:00002fcc       $unwind$check_option       0000000180008fcc     libthrcputime002.obj
 0002:00002fcc       $unwind$nsk_jvmti_findOptionValue 0000000180008fcc     libthrcputime002.obj
 0002:00002fcc       $unwind$_DllMainCRTStartup 0000000180008fcc     MSVCRT:dll_dllmain.obj
 0002:00002fdc       $unwind$nsk_jvmti_findOptionIntValue 0000000180008fdc     libthrcputime002.obj
 0002:00002fec       $unwind$nsk_jvmti_lverify  0000000180008fec     libthrcputime002.obj
 0002:00003000       $unwind$exitOnError        0000000180009000     libthrcputime002.obj
 0002:00003010       $unwind$Java_nsk_share_jvmti_ArgumentHandler_getAgentOptionsString 0000000180009010     libthrcputime002.obj
 0002:00003024       $unwind$Java_nsk_jvmti_unit_FollowReferences_FollowRefObjects_getTag 0000000180009024     libthrcputime002.obj
 0002:00003024       $unwind$Java_nsk_share_jvmti_DebugeeClass_checkStatus 0000000180009024     libthrcputime002.obj
 0002:00003024       $unwind$agentThreadWrapper 0000000180009024     libthrcputime002.obj
 0002:00003034       $unwind$startAgentThreadWrapper 0000000180009034     libthrcputime002.obj
 0002:00003050       $unwind$syncDebuggeeStatus 0000000180009050     libthrcputime002.obj
 0002:00003050       $unwind$__scrt_dllmain_exception_filter 0000000180009050     MSVCRT:utility.obj
 0002:00003064       $unwind$Java_nsk_share_jvmti_DebugeeClass_resetAgentData 0000000180009064     libthrcputime002.obj
 0002:0000306c       $unwind$MA_checkStatus     000000018000906c     libthrcputime002.obj
 0002:00003080       $unwind$Java_nsk_jvmti_unit_FollowReferences_FollowRefObjects_setTag 0000000180009080     libthrcputime002.obj
 0002:00003098       $unwind$Java_nsk_jvmti_unit_FollowReferences_FollowRefObjects_addRefToVerify 0000000180009098     libthrcputime002.obj
 0002:000030b4       $unwind$Agent_Initialize   00000001800090b4     libthrcputime002.obj
 0002:000030d8       $unwind$checkCpuTime       00000001800090d8     libthrcputime002.obj
 0002:000030f8       $unwind$agentProc          00000001800090f8     libthrcputime002.obj
 0002:00003110       $unwind$callbackVMInit     0000000180009110     libthrcputime002.obj
 0002:00003124       $unwind$callbackThreadStart 0000000180009124     libthrcputime002.obj
 0002:0000313c       $unwind$callbackThreadEnd  000000018000913c     libthrcputime002.obj
 0002:00003158       $unwind$capture_previous_context 0000000180009158     MSVCRT:gs_report.obj
 0002:00003164       $unwind$__GSHandlerCheckCommon 0000000180009164     MSVCRT:gshandler.obj
 0002:00003170       $xdatasym                  0000000180009170     MSVCRT:amdsecgs.obj
 0002:00003174       $unwind$?dllmain_crt_process_attach@@YAHQEAUHINSTANCE__@@QEAX@Z 0000000180009174     MSVCRT:dll_dllmain.obj
 0002:000031b0       $unwind$?fin$0@?0??dllmain_crt_process_attach@@YAHQEAUHINSTANCE__@@QEAX@Z@4HA 00000001800091b0     MSVCRT:dll_dllmain.obj
 0002:000031b0       $unwind$?fin$0@?0??dllmain_crt_process_detach@@YAH_N@Z@4HA 00000001800091b0     MSVCRT:dll_dllmain.obj
 0002:000031b0       $unwind$?fin$1@?0??dllmain_crt_process_detach@@YAH_N@Z@4HA 00000001800091b0     MSVCRT:dll_dllmain.obj
 0002:000031b8       $unwind$?dllmain_crt_process_detach@@YAH_N@Z 00000001800091b8     MSVCRT:dll_dllmain.obj
 0002:0000320c       $unwind$?dllmain_dispatch@@YAHQEAUHINSTANCE__@@KQEAX@Z 000000018000920c     MSVCRT:dll_dllmain.obj
 0002:00003234       $unwind$?filt$0@?0??dllmain_dispatch@@YAHQEAUHINSTANCE__@@KQEAX@Z@4HA 0000000180009234     MSVCRT:dll_dllmain.obj
 0002:0000323c       $unwind$__scrt_is_nonwritable_in_current_image 000000018000923c     MSVCRT:utility.obj
 0002:0000325c       $unwind$__scrt_is_nonwritable_in_current_image$filt$0 000000018000925c     MSVCRT:utility.obj
 0002:00003264       $unwind$__scrt_fastfail    0000000180009264     MSVCRT:utility_desktop.obj
 0002:00003274       $unwind$__security_init_cookie 0000000180009274     MSVCRT:gs_support.obj
 0002:00003280       $unwind$__isa_available_init 0000000180009280     MSVCRT:cpu_disp.obj
 0002:00003290       $xdatasym                  0000000180009290     MSVCRT:guard_dispatch.obj
 0002:00003298       $xdatasym                  0000000180009298     MSVCRT:guard_xfg_dispatch.obj
 0002:000032a0       .edata                     00000001800092a0     thrcputime002.exp
 0002:000032c8       rgpv                       00000001800092c8     thrcputime002.exp
 0002:00003310       rgszName                   0000000180009310     thrcputime002.exp
 0002:00003358       rgwOrd                     0000000180009358     thrcputime002.exp
 0002:0000337c       szName                     000000018000937c     thrcputime002.exp
 0002:0000338e       $N00001                    000000018000938e     thrcputime002.exp
 0002:0000339d       $N00002                    000000018000939d     thrcputime002.exp
 0002:000033aa       $N00003                    00000001800093aa     thrcputime002.exp
 0002:000033ef       $N00004                    00000001800093ef     thrcputime002.exp
 0002:0000342c       $N00005                    000000018000942c     thrcputime002.exp
 0002:00003474       $N00006                    0000000180009474     thrcputime002.exp
 0002:000034b4       $N00007                    00000001800094b4     thrcputime002.exp
 0002:000034f1       $N00008                    00000001800094f1     thrcputime002.exp
 0002:0000352c       $N00009                    000000018000952c     thrcputime002.exp
 0002:0000355a       $N00010                    000000018000955a     thrcputime002.exp
 0002:0000358b       $N00011                    000000018000958b     thrcputime002.exp
 0002:000035ba       $N00012                    00000001800095ba     thrcputime002.exp
 0002:000035e9       $N00013                    00000001800095e9     thrcputime002.exp
 0002:0000361e       $N00014                    000000018000961e     thrcputime002.exp
 0002:0000362d       $N00015                    000000018000962d     thrcputime002.exp
 0002:0000363f       $N00016                    000000018000963f     thrcputime002.exp
 0002:00003653       $N00017                    0000000180009653     thrcputime002.exp
 0002:00003663       $N00018                    0000000180009663     thrcputime002.exp
 0002:00003aca       .idata$6                   0000000180009aca     kernel32:KERNEL32.dll
 0002:00003b2e       .idata$6                   0000000180009b2e     vcruntime:VCRUNTIME140.dll
 0002:00003cc0       .idata$6                   0000000180009cc0     ucrt:api-ms-win-crt-heap-l1-1-0.dll
 0002:00003ce0       .idata$6                   0000000180009ce0     ucrt:api-ms-win-crt-runtime-l1-1-0.dll
 0002:00003d02       .idata$6                   0000000180009d02     ucrt:api-ms-win-crt-convert-l1-1-0.dll
 0002:00003d24       .idata$6                   0000000180009d24     ucrt:api-ms-win-crt-stdio-l1-1-0.dll
 0002:00003d44       .idata$6                   0000000180009d44     ucrt:api-ms-win-crt-string-l1-1-0.dll
 0003:00000000       ?codeAttributeName@@3PEBDEB 000000018000a000     libthrcputime002.obj
 0003:00000008       ?lineNumberAttributeName@@3PEBDEB 000000018000a008     libthrcputime002.obj
 0003:00000010       ?localVarAttributeName@@3PEBDEB 000000018000a010     libthrcputime002.obj
 0003:00000018       ?localVarTypeAttributeName@@3PEBDEB 000000018000a018     libthrcputime002.obj
 0003:00000020       ?stackMapAttributeName@@3PEBDEB 000000018000a020     libthrcputime002.obj
 0003:00000028       ?callBytes@@3PAEA          000000018000a028     libthrcputime002.obj
 0003:0000002c       ?allocBytes@@3PAEA         000000018000a02c     libthrcputime002.obj
 0003:00000030       events                     000000018000a030     libthrcputime002.obj
 0003:00000038       threadEvents               000000018000a038     libthrcputime002.obj
 0003:0001aae4       redefineAttempted          0000000180024ae4     libthrcputime002.obj
 0003:0001aae8       nsk_context                0000000180024ae8     libthrcputime002.obj
 0003:0001aaf4       redefineSucceed            0000000180024af4     libthrcputime002.obj
 0003:0001aaf8       agentFailed                0000000180024af8     libthrcputime002.obj
 0003:0001aafc       currentAgentStatus         0000000180024afc     libthrcputime002.obj
 0003:0001ab00       context                    0000000180024b00     libthrcputime002.obj
 0003:0001abb8       agentThread                0000000180024bb8     libthrcputime002.obj
 0003:0001abc0       agentThreadProc            0000000180024bc0     libthrcputime002.obj
 0003:0001abc8       agentThreadArg             0000000180024bc8     libthrcputime002.obj
 0003:0001abd0       agent_data                 0000000180024bd0     libthrcputime002.obj
 0003:0001abe0       jvmti_env                  0000000180024be0     libthrcputime002.obj
 0003:0001abe8       jvm                        0000000180024be8     libthrcputime002.obj
 0003:0001abf0       jni_env                    0000000180024bf0     libthrcputime002.obj
 0003:0001abf8       checkStatus_func           0000000180024bf8     libthrcputime002.obj
 0003:0001ac00       ?codeAttributeIndex@@3GA   0000000180024c00     libthrcputime002.obj
 0003:0001ac04       ?lineNumberAttributeIndex@@3GA 0000000180024c04     libthrcputime002.obj
 0003:0001ac08       ?localVarAttributeIndex@@3GA 0000000180024c08     libthrcputime002.obj
 0003:0001ac0c       ?localVarTypeAttributeIndex@@3GA 0000000180024c0c     libthrcputime002.obj
 0003:0001ac10       ?stackMapAttributeIndex@@3GA 0000000180024c10     libthrcputime002.obj
 0003:0001ac14       ?stackFrameOffset@@3GA     0000000180024c14     libthrcputime002.obj
 0003:0001ac18       ?mode@@3HA                 0000000180024c18     libthrcputime002.obj
 0003:0001ac1c       ?constantPoolSize@@3GA     0000000180024c1c     libthrcputime002.obj
 0003:0001ac20       ?orig@@3PEBEEB             0000000180024c20     libthrcputime002.obj
 0003:0001ac28       ?gen@@3PEAEEA              0000000180024c28     libthrcputime002.obj
 0003:0001ac30       ?inputPos@@3PEAEEA         0000000180024c30     libthrcputime002.obj
 0003:0001ac38       ?endPos@@3PEBEEB           0000000180024c38     libthrcputime002.obj
 0003:0001ac40       ?genPos@@3PEAEEA           0000000180024c40     libthrcputime002.obj
 0003:0001ac48       ?markPos@@3PEAEEA          0000000180024c48     libthrcputime002.obj
 0003:0001ac50       ?constantPool@@3PEAPEADEA  0000000180024c50     libthrcputime002.obj
 0003:0001ac58       ?constantPoolCount@@3GA    0000000180024c58     libthrcputime002.obj
 0003:0001ac5c       ?zeroBytes@@3PAEA          0000000180024c5c     libthrcputime002.obj
 0003:0001ac60       ?codeLength@@3IA           0000000180024c60     libthrcputime002.obj
 0003:0001ac64       iterations                 0000000180024c64     libthrcputime002.obj
 0003:0001ac68       ?map@@3PEAIEA              0000000180024c68     libthrcputime002.obj
 0003:0001ac70       ?widening@@3PEACEA         0000000180024c70     libthrcputime002.obj
 0003:0001ac78       timeout                    0000000180024c78     libthrcputime002.obj
 0003:0001ac80       monitor                    0000000180024c80     libthrcputime002.obj
 0003:0001ac88       prevTestedThreadTime       0000000180024c88     libthrcputime002.obj
 0003:0001ac90       prevAgentThreadTime        0000000180024c90     libthrcputime002.obj
 0003:0001ac98       testedThread               0000000180024c98     libthrcputime002.obj
 0003:0001aca0       testAgentThread            0000000180024ca0     libthrcputime002.obj
 0003:0001acb0       GS_ExceptionRecord         0000000180024cb0     MSVCRT:gs_report.obj
 0003:0001ad50       GS_ContextRecord           0000000180024d50     MSVCRT:gs_report.obj
 0003:0001b220       ?g_tss_cv@@3U_RTL_CONDITION_VARIABLE@@A 0000000180025220     MSVCRT:thread_safe_statics.obj
 0003:0001b228       ?g_tss_event@@3PEAXEA      0000000180025228     MSVCRT:thread_safe_statics.obj
 0003:0001b230       ?g_tss_mutex@@3U_RTL_CRITICAL_SECTION@@A 0000000180025230     MSVCRT:thread_safe_statics.obj
 0003:0001b258       ?g_sleep_condition_variable_cs@@3P6AHPEAU_RTL_CONDITION_VARIABLE@@PEAU_RTL_CRITICAL_SECTION@@K@ZEA 0000000180025258     MSVCRT:thread_safe_statics.obj
 0003:0001b260       ?g_wake_all_condition_variable@@3P6AXPEAU_RTL_CONDITION_VARIABLE@@@ZEA 0000000180025260     MSVCRT:thread_safe_statics.obj
 0003:0001b26c       ?__proc_attached@@3HA      000000018002526c     MSVCRT:dll_dllmain.obj
 0003:0001b280       ?is_initialized_as_dll@@3_NA 0000000180025280     MSVCRT:utility.obj
 0003:0001b281       ?module_local_atexit_table_initialized@@3_NA 0000000180025281     MSVCRT:utility.obj
 0003:0001b288       ?module_local_atexit_table@@3U_onexit_table_t@@A 0000000180025288     MSVCRT:utility.obj
 0003:0001b2a0       ?module_local_at_quick_exit_table@@3U_onexit_table_t@@A 00000001800252a0     MSVCRT:utility.obj
